:100000000C9466000C9487000C9487000C94870075
:100010000C9487000C9487000C9487000C94870044
:100020000C9487000C9487000C9487000C94870034
:100030000C9487000C9487000C9487000C94870024
:100040000C9487000C9487000C9487000C94870014
:100050000C9487000C9458030C9487000C94870030
:100060000C9487000C943E130C9487000C9487002A
:100070000C9487000C9487000C9487000C948700E4
:100080000C94A0000C9487000C9487000C948700BB
:100090000C942B1B0C9487000C9487000C94870005
:1000A0000C9487000C9487000C9487000C948700B4
:1000B0000C9487000C9487000C9487000C948700A4
:1000C0000C9487000C9487000C94870011241FBEA9
:1000D000CFEFD1E2DEBFCDBF00E00CBF14E0A0E067
:1000E000B2E0EAEDF4E900E00BBF02C007900D9228
:1000F000A434B107D9F717E0A4E4B4E001C01D921D
:10010000AA33B107E1F70E94EF0C0C946B4A0C94F0
:1001100000001092550410924A0480914A04809382
:100120004904809149048093480480914804809355
:10013000470410924B0410925804109259040895E9
:100140001F920F920FB60F9211240F900FBE0F90B7
:100150001F901895EEE6F0E080818260808383E056
:1001600084BD85BD8AEF87BD08951092900088E018
:10017000809391008BE09AE190939900809398008E
:10018000109295001092940082E08093710008957F
:100190000895089580917100817008959B01AC01CC
:1001A000CA01AA27BB27BC01892B79F0687F672B7E
:1001B00059F483E056954795379527958A95D1F759
:1001C0003093AE042093AD0408953093AE04209391
:1001D000AD0408958091AB04982F929596959695CD
:1001E0009370282F221F2227221F9227282F229523
:1001F0002F709227282F2695269592279170880F89
:10020000892B8093AB04089590939D0480939C0464
:1002100085EB9BE39093B5048093B40483E393E16F
:100220009093BB048093BA0485E694ED9093B00458
:100230008093AF04089580919C0490919D04AC013B
:10024000440F452F441F550B51954827592760915E
:10025000B4047091B50470939D0460939C048091E4
:10026000BA049091BB049093B5048093B404209198
:10027000AF043091B0043093BB042093BA04C90199
:100280000024969587950794969587950794982FBF
:10029000802D8227932784279527542F4427529512
:1002A000550F507E842795279093B0048093AF0418
:1002B000660F771F6F5F7F4F869F9001879F300D7E
:1002C000969F300D1124C9010895FC019081992356
:1002D00051F08091C80085FFFCCF9093CE003196FD
:1002E00090819923B1F708951F93CF93DF93182F2F
:1002F000492FE0E1F7E2C0E0D0E0812F942FBF0169
:100300000E94224A9B016115710589F5812F942F66
:10031000BF010E94224A182F492FCF016AE070E0E6
:100320000E94224AFB012196C430D10531F7309753
:10033000A1F18091C80085FFFCCF812F942FBF01D0
:100340000E94224A605D6093CE00CF016AE070E0B7
:100350000E94224A9B0161157105F9F0812F942FAB
:10036000BF010E94224A182F492FF901E2CF809144
:10037000C80085FFFCCF822F805D8093CE00812F47
:10038000942FBF010E94224A182F492FCF016AE003
:1003900070E00E94224AFB01CACFDF91CF911F91EA
:1003A0000895982F9F709A3040F48091C80085FF7F
:1003B000FCCF905D9093CE0008958091C80085FF9A
:1003C000FCCF995C9093CE000895CF93DF93EC011E
:1003D000892F992782958F700097C1F48D2F9927C7
:1003E000009789F4CE01929582958F7089279F702E
:1003F0008927009711F00E94D1018C2F0E94D10112
:10040000DF91CF9108950E94D101ECCF0E94D101DC
:10041000E5CF982F8091C80085FFFCCF9093CE0048
:1004200080E090E008952091C800332727FD3095A3
:100430002227330F221F3327C90108958091C80056
:1004400087FFFCCF8091CE0090E008959C018FEF54
:100450008093A10493E0283E390768F580939E04B9
:1004600080939F0424363105D8F0C90164E670E01A
:100470000E94224A60939E04C9016AE070E00E94D3
:10048000224ACB016AE070E00E94224A80939F04D6
:10049000C9016AE070E00E94224A8093A004089596
:1004A0002A30310548F7C9016AE070E00E94224A0B
:1004B0008093A004089510929E0410929F041092BD
:1004C000A004089590914C04936090934C04809301
:1004D0004D04089580914C04836080934C040895EA
:1004E000F999FECF92BD81BDF89A30B5F999FECF4A
:1004F000019692BD81BDF89A20B5932F80E030E03F
:10050000282B392BC9010895F999FECF92BD81BDE1
:10051000F89A80B50895F999FECF92BD81BD60BD6E
:10052000F894FA9AF99A78940895FF920F931F938A
:100530008C01F62E672F0E948B02C80101966F2D49
:100540000E948B021F910F91FF9008958091C90026
:1005500088618093C90083E38093CC001092CD0022
:100560008091C80087FD34C08091C9008068809365
:10057000C9008091C10088698093C1008FE1809398
:10058000C4001092C50090EC91B98CE382B987E366
:1005900084B995B99FEF97B988EF8AB98BE08BB989
:1005A00082E08DB99EB910BA91BB88E183BB87EE1A
:1005B00084BB8DB581608DBD81E58CBD0895809132
:1005C000CE008AE00E94A20F8091C80087FFCCCFA6
:1005D0008091C80087FDF3CF8091C80087FFF8CFD6
:1005E000EECFEF92FF920F931F93CF93DF93EC0127
:1005F00081E0CD32D80708F440C0CCE2D1E07E01E2
:1006000000E010E080919804909199048C179D0768
:1006100019F0CE010E94E61AD0939904C093980471
:10062000D093AA04C093A9046091090270910A02B0
:1006300080910B0290910C02A80197010E94494AF7
:100640006FEF7FEF8FEF9FEF0E94494ACA01B90118
:1006500028EE33E040E050E00E94F7496093A504A3
:100660007093A6048093A7049093A804DF91CF9180
:100670001F910F91FF90EF900895C431D10508F0BC
:10068000BECFC4E1D0E054E1E52EF12C012D112DB7
:10069000B9CF85E090E00E9470020E94F102809143
:1006A0009804909199049093B2048093B1040895B2
:1006B0001F920F920FB60F920BB60F9211242F9329
:1006C0003F934F935F936F937F938F939F93AF93DA
:1006D000BF93EF93FF9340B1427090B18091B80403
:1006E000481749F1892F8170442309F4D8C0882321
:1006F00009F4D8C09FEF809101048823D1F0809144
:100700005304882309F4FAC0913009F017C180918D
:10071000A9049091AA0407969093AA048093A9042F
:100720008D52914030F08CE291E09093AA04809336
:10073000A9044093B804809168048F3F29F0809108
:1007400068048F5F80936804809169048F3F29F06B
:10075000809169048F5F8093690480917704909100
:1007600078048F5F9F4F49F08091770490917804CF
:10077000019690937804809377048091560488239F
:1007800051F0809156048150809356048091560414
:10079000882309F49AC080919304909194048F5F08
:1007A0009F4F49F080919304909194040196909307
:1007B00094048093930480914404823009F487C0A8
:1007C000813009F471C0882309F056C0809101027C
:1007D00090910202A0910302B0910402809305025D
:1007E00090930602A0930702B093080220910102A1
:1007F0003091020240910302509104028091A504BD
:100800009091A604A091A704B091A804820F931F11
:10081000A41FB51F8093010290930202A0930302CC
:10082000B093040220910102309102024091030230
:10083000509104028091050290910602A091070256
:10084000B0910802281739074A075B07A8F480917E
:1008500055048F5F80935504809155048170809377
:100860005504809154048F5F809354048091A904AF
:100870009091AA040E94F102FF91EF91BF91AF9174
:100880009F918F917F916F915F914F913F912F91A8
:100890000F900BBE0F900FBE0F901F9018958823DE
:1008A00009F428CF91E027CF99B19295917080916A
:1008B0006604981709F39093550490936604809109
:1008C00054048F5F80935404D7CFA49864CF809151
:1008D000620490916304892B79F280916204909173
:1008E000630401979093630480936204809162048F
:1008F00090916304892B09F0BFCFE1CF292F3327D3
:1009000027FD30958091A9049091AA04280F391FE2
:100910003093AA042093A90481E02D32380708F00F
:1009200002CF2431310508F004CF84E190E09093A8
:10093000AA048093A9044093B804FDCE9F3F09F018
:10094000F8CE8091A9049091AA0407979093AA04E5
:100950008093A904449708F0ECCEE7CFCF92DF92C2
:10096000EF92FF920F931F93CF93DF93F8948091B0
:100970004404813009F4C7C480918F04813009F4A4
:10098000DFC2809147048C3060F010924704809160
:1009900048048F5F80934804809149048F5F80935F
:1009A000490480914904882341F08091490490E0F2
:1009B00083709070892B09F45CC280914A0488305E
:1009C00038F010924A0480914404882309F430C21C
:1009D000809149048F7080934904909148048091DC
:1009E00000029817C0F01092480480914B048F5F6A
:1009F00080934B0490914B048091B904981708F0B0
:100A000014C280914C04826080934C048091500405
:100A100081608093500480913407882329F4809169
:100A20004804882309F4F7C180914804882329F4F5
:100A300080918F04823009F4A3C290915804809170
:100A4000B304981710F0109258048091340788234B
:100A500029F080915804882309F411C28091F70489
:100A60008C3009F415C280914404882309F005C133
:100A7000909161048091FF03981710F01092610427
:100A80008091610480FFF3C05C9880919004209174
:100A9000FF034091FF0390E030E0240F311D8217E7
:100AA000930714F010929004E091FF03E695E69509
:100AB000E69520915A0490919004E150F0E0EE0FF9
:100AC000FF1FEE0FFF1FE20FF11DE35FFD4F80815F
:100AD000891709F4F9C1DD248091FF03869590916F
:100AE000AC04899F902D112480915904891710F02E
:100AF0001092590480913407882349F08091590459
:100B0000882309F4A39A9695891709F449C280911C
:100B1000F704873009F4D3C0883008F4C8C08B309C
:100B200009F4CDC08C3008F43DC28C3009F46DC39B
:100B30008D3009F4C4C080918F04823009F4FBC366
:100B400080913407882321F082E0D81609F4FEC38F
:100B500080913407882309F403C280917C048F704C
:100B600080937C048091490490E083709070029798
:100B70000CF4F2C185E20E94FF1680917C0490E0A3
:100B80008370907002970CF4E4C18FEF809374042B
:100B900080918504882309F0A3C180918E04882365
:100BA00071F080914D04882351F08091B60481301A
:100BB00009F42BC28091B604882309F416C28091EF
:100BC0004E04813009F4E4C3823009F4C3C3809138
:100BD0005304882349F080914404882329F48091A8
:100BE0000104882309F021C20E94D618DD2031F0CB
:100BF000809145048F5F81708093450480919004BB
:100C00008F5F80939004809128078F5F80932807DF
:100C1000809147048F5F80934704809161048F5FC8
:100C200080936104809158048F5F80935804809171
:100C300059048F5F80935904209128078091FF0306
:100C400030E086958695869548E1849FC001112401
:100C50002817390714F0109228077894DF91CF9164
:100C60001F910F91FF90EF90DF90CF9008955C9AC5
:100C700088EF0E94AD1080914404813009F419C1BD
:100C8000823009F002CF809155048F5F8093550424
:100C90008091550481708093550480915504882378
:100CA00009F4F2CE5C9A88EF0E94AD10EECE81304E
:100CB00008F441CF843018F0853009F03CCF81E052
:100CC000D81609F4E8C1E2E0DE1609F034CF8091CD
:100CD0007C048F5F80937C0480913407882309F41F
:100CE00094C08091BB05882309F510922807809154
:100CF000BF05882349F480912A07882329F0809131
:100D00008504882309F025C68091430660918B06EF
:100D1000680F8091CF069091D0060E94AA2A109267
:100D20007C0480918004882309F440C58091BB0530
:100D3000E091CF06F091D006E80FF11D80818093FD
:100D400097048091A4048093A204809197048074F6
:100D50008093A40480918504882309F0C5C4809100
:100D600097048F708F3009F417C5809197048F70A6
:100D70008F3029F1809197040E94CE2A0091D506E8
:100D8000080F1091970410786091A204802F412FD2
:100D90000E94401E112309F007C580E0902F935F49
:100DA000982B80915104981751F0809151048093B1
:100DB000520490935104809151040E9461108091DB
:100DC000F704833009F483C48091F7048730E9F491
:100DD00080914E04882309F0AFC58091A3059091BE
:100DE000A405E091B405F0E0EE0FFF1FEB5EFD4FB0
:100DF0006081718182959295907F9827807F982756
:100E00000E94224A862F0E94AF1780914C04816075
:100E100080934C0490CE80918F04823009F004CEF0
:100E200010928F040E94CF33FFCD10924B04E9CD76
:100E300020919804309199048091B1049091B2046A
:100E40002817390709F4C4CD80913407882309F0A5
:100E5000BFCD85E20E94C7166091980470919904F5
:100E60007093B2046093B10485E090E00E94950213
:100E7000AFCD80914A048F5F80934A049ECDA49A9F
:100E800085E0809356048091F7048C3009F0EBCD17
:100E90008091500480FF0AC080913407882309F0B4
:100EA00080C280915D04882309F084C310925004AD
:100EB000DACD80915504882309F4E7CD88EF0E94AC
:100EC000AD1080914404DCCE2F5F237020935A0430
:100ED00080914504882309F450C0DD24D394FCCDCF
:100EE0008CE20E94CE2A982F80917C048111945F1D
:100EF00080912807882341F480918604882309F48F
:100F0000A1C383E20E94C71680912807843009F0AC
:100F100044CE80918604882379F4809183048230C2
:100F200008F4AFC3809147060E94CE2A409147063D
:100F3000407860E00E94401E83E20E94FF162DCEA2
:100F400080913407882381F00E94CB2E10928F0469
:100F500018CD109274041CCE85E20E94C7160DCEE7
:100F600081E20E94FF16F9CD0E94CF3380914404A4
:100F7000882361F70E948900E9CF52E0D52EACCDDD
:100F80008091F704853009F458CD10925A041092DC
:100F90009004109245041092BB0510928F044DCD21
:100FA000A398B5CD883009F0C6CDF1E0DF1609F47D
:100FB0004FC382E0D81609F0BECD8091960480938D
:100FC000460480919504809396040E94EA008093E1
:100FD0009504809196048F7360E040E00E94401E6B
:100FE000809196040E946110A6CD80914C0480FFF0
:100FF000E6CD80914C048E7F80934C040E948B1729
:101000008091BB050E949917DACD80914C0481FF35
:10101000D1CD80914C048D7F80934C040E948B171E
:1010200080914B040E949917C5CD0E948B17609147
:10103000980470919904603A710508F48AC2603A84
:10104000710509F42BC380E090E02EE030E040E031
:1010500050E00E94F749685E7E4F8F4F9F4F28E116
:1010600031E040E050E00E94494A022F293008F464
:101070006BC418E0812F0E9499171F5F1017D0F3DF
:10108000003108F0B1CD102F812F0E94A4171F5FEF
:101090001031D0F3A9CD8091BF058F5F8093BF053C
:1010A00080913407882309F446CD8091BB058F5F7A
:1010B0008093BB059091BB0580910004981710F0B8
:1010C0001092BB058091BB05882309F06EC080910A
:1010D000F704833009F49BC210E08091F704873055
:1010E00009F414C381E00E94792A80918B068F5FF6
:1010F00080938B06C0908B0690918B068091490659
:10110000981708F443C080918004882319F481E083
:1011100080938D048091F704813009F462C380913B
:10112000F704823009F459C382E00E94792A1092B0
:10113000BF0580918504882369F0809183048093A2
:101140002A0780912A07882329F01092830481E0DE
:101150008093B90510928B068091F704833009F4CF
:1011600093C38091F704873009F452C380914A06F3
:10117000882309F039C3909127078091BA05981701
:1011800029F080918004823008F417C480918B0686
:1011900090E082959295907F9827807F982783573B
:1011A000994F9093D0068093CF0680918504882331
:1011B00009F0C1CC8091BB05E091CF06F091D0063B
:1011C000E80FF11D808180939704809197048F70C0
:1011D0008F3009F4DEC28091A4040E94571E8091D2
:1011E0005204882309F0CEC28091A404882309F018
:1011F000A2CC80915104882309F49DCC80915104A4
:101200000E9487101092510496CC0E948B178091F7
:10121000500480FD16C180915D04882309F00BC144
:10122000E1E0DE1609F411C1F2E0DF1609F083CC2B
:1012300080917C048F5F80937C04809134078823A5
:1012400009F479CCE0918B06F0E0EF52F94F808100
:1012500084FD22C28CE08093FF038091BB05E09166
:10126000CF06F091D006E80FF11D8081809397049E
:101270008091A4048093A204809197048074809349
:10128000A404809197048F708F3009F418C2809164
:1012900097048F708F3071F0809197040E94CE2A4E
:1012A0009091D5066091A204409197044078890FEF
:1012B0000E94401E80914F04982F92959F709093AA
:1012C000E606982F977090934306869586958695A7
:1012D00081708093270780912707882309F0D5C163
:1012E00088E00E94C71681E00E94FF160E947F18C6
:1012F000809143068F5F0E941F1880913407817090
:101300008093340718CC0E94D713882339F080913A
:101310008E04882309F0AAC10E9489000E94E91363
:10132000882309F429CB80918E04882309F424CBE7
:101330000E94CB2E21CB81E20E94FF1680914704B0
:1013400063E00E94164A992309F007CC81E20E94CB
:10135000C71603CC0E947D1A90919E04892F81505C
:10136000823008F47FC190919F048091A004981767
:1013700009F4D8C0992319F0892F0E94721A80911C
:10138000490481FF24CC8091A0040E94721A1FCCD2
:101390000E947D1A8091490480FFCFC080914E0445
:1013A00013CC80913407823008F480CD80915D04A5
:1013B000882329F48091A705882309F477CD8091AB
:1013C0005E0480934F0490918B069F5F90938B06F1
:1013D00090918B06917090938B0660918B0670E0D4
:1013E00062957295707F7627607F76276357794F75
:1013F0007093D0066093CF0690918B06C92FD0E0F2
:101400000E94142DCF52D94F8883E0918B06F0E0D3
:10141000EF52F94F80818F708F5F80930004E091CD
:101420008B06F0E0EF52F94F808184FD19C18CE00A
:101430008093FF033BCD80915D0481500E949917FA
:10144000EFCE8FE00E949917E6CE80913407882373
:1014500009F471CB8091BB058F5F8093BB058091B0
:101460005D04882309F405C190915E0480914F04C6
:101470008917D1F1F0908B06F394FE220F2D10E026
:10148000E801C295D295D07FDC27C07FDC27C35707
:10149000D94F80915E04BE010E94142D0F52194F46
:1014A000F8018083E0918B06F0E0EF52F94F208144
:1014B000F801808190E030E08227932784FD14C0FA
:1014C00080915E0480934F04F0928B06E0918B062E
:1014D000F0E0EF52F94F80818F708F5F80930004AE
:1014E000D093D006C093CF068091BB0560910004D5
:1014F0000E94164A9093BB058091BB05E091CF06F0
:10150000F091D006E80FF11D8081809397048091BF
:1015100097048F708F3009F4CAC08091A4040E9490
:10152000571E09CB992309F42ACF8091490482FFE1
:101530004ECB892F0E94721A4ACBE0914904E6955E
:10154000F0E0E370F070E256FB4F80810E94721A67
:1015500025CF80E090E02EE030E040E050E00E94B7
:10156000F7496E5070408040904028E131E040E003
:1015700050E00E94494A022F222309F42CC110E0B6
:10158000812F0E94A4171F5F1017D0F3083008F0B6
:1015900020C1102F812F0E9499171F5F1830D0F3A0
:1015A000103108F021CB812F0E94A4171F5F10314A
:1015B000D0F31ACB80915E0480934F040E94CF3306
:1015C00080914404882309F49EC010925A048091AB
:1015D0008B068F5F80938B0680918B068170809342
:1015E0008B0660918B0670E062957295707F76270E
:1015F000607F76276357794F7093D0066093CF064C
:1016000080918B06C82FD0E080914F04F9CE809155
:10161000A3059091A40501969093A4058093A3053A
:101620002091A3053091A4058091AE059091AF055E
:101630002817390708F450CD1092A4051092A3057D
:1016400011E04BCD892F60E040E00E94401E59CC54
:1016500080E00E94571E809196040E9487106BCAFA
:1016600080E1E6CE865F0E94721A7DCE0E94CF3363
:1016700053CE8091A705882309F036CF0E94CB2E48
:1016800033CF80E00E94571E57CC88E00E94FF169F
:1016900081E00E94C7162ACE80E1DDCD0E948B1723
:1016A00087E00E94991788E00E9499179DCA80914F
:1016B000A404882309F089C01092A4042ECF80913D
:1016C00097048F70809397041092A404E0CD8091CA
:1016D0004E04882309F478CB8091A3059091A4054A
:1016E00001960E94260270CB8091430660914906C4
:1016F0004091BC0520914A060091C005E090BA05D2
:101700000E94C5195CCB0E9489005FCF80917B0449
:10171000813009F0E7CC6091270780914306409122
:101720008B062091D506480F8BEA95E00E94C11FD9
:101730008091B4056091A3057091A4054091AB051B
:101740000E94CF208091A3059091A40501969093CB
:10175000A4058093A305E091B4052091A3053091E1
:10176000A405F0E0EE0FFF1FEB5EFD4F808191813D
:101770002817390708F4B6CC10927B0483E20E9444
:10178000FF16B0CC809152040E9487101092520430
:101790002BCD1092A4041FCD809197048F7080935D
:1017A00097041092A404E1CA80E8F8CA8091430625
:1017B000609149064091BC0520914A060091C00500
:1017C000E090BA050E94C519B1CA81E00E94571E77
:1017D00073CF102FE5CE10E0DDCE81E080938D0435
:1017E000A3CC80938D049BCC0E94662A80918004B8
:1017F000823008F0CBCC8091E606609127074091BB
:101800004306209149060DE816E00E94712DBECCDA
:1018100080917B04813009F0A9CC8091A7058823B1
:10182000B9F010927B041092A7058091B4056091E5
:10183000A3057091A4050E94A6208091B4050E9482
:1018400032219093AF058093AE0583E20E94FF168C
:101850008091A805882309F489CC1092A80580916D
:10186000B4056091A3057091A4056C190E9496209F
:101870008091B4050E9429219093B6058093B50507
:1018800080E00E94FF1672CC8091A705882309F0A2
:101890007BC08091A805882309F458C01092A40544
:1018A0001092A3058091F2048093B4058091B40551
:1018B0000E9432219093AF058093AE058091B405CC
:1018C0000E9429219093B6058093B5052091B50516
:1018D0003091B6058091AE059091AF052817390774
:1018E00020F01092B6051092B5058091A8058823C6
:1018F00009F055C08091B4056091A3057091A405CD
:101900000E9483218093AB058091B4056091AB0563
:1019100042E056E02AEB35E00CEB15E09EECE92EB8
:1019200096E0F92E0E94A11F81E080934A068091E3
:10193000CE068093D50615CC8091A3059091A40581
:1019400001960E94260249CA18E09ECB112369F233
:10195000A5CF81E00E94571E80E00E94571E609133
:1019600049068DE896E047EE56E021EC35E00E940E
:10197000D92B109285048AE00E94EA2A1092A404CE
:1019800082E00E94A20FC0C91092A7051092A40580
:101990001092A30583E20E94FF1611E07ACF109205
:1019A000A8058091B5059091B6059093A405809304
:1019B000A30580E00E94FF169DCF8091BA05809319
:1019C000270719CF07C08091540481508093540495
:1019D0000E94AE04809154048823A9F70895AF9221
:1019E000BF92CF92DF92EF92FF920F931F93DF93FC
:1019F000CF93CDB7DEB760970FB6F894DEBF0FBEBA
:101A0000CDBF0E94A6020E94490380916E008260B1
:101A100080936E0083E084BD85BD8AEF87BD8DE82D
:101A200096E09093D0068093CF06F999FECF82E09E
:101A300090E092BD81BDF89A80B5982F93709093F5
:101A400044048295817080938604F999FECF87E0E3
:101A500090E092BD81BDF89A80B5882311F0813263
:101A600008F080E180930002F999FECF83E090E0D6
:101A700092BD81BDF89A80B58F708093CF04F9999B
:101A8000FECF84E090E092BD81BDF89A80B58F7062
:101A90008093BC0488E090E00E9470028093AB04C5
:101AA0002091980430919904280F391F30939D0498
:101AB00020939C0485EB9BE39093B5048093B4043E
:101AC00083E393E19093BB048093BA0485E694ED9D
:101AD0009093B0048093AF040E941B010E941B01ED
:101AE0000E941B01BC0188E090E00E949502F999D8
:101AF000FECF8AE090E092BD81BDF89A90B5892F23
:101B00008F708093B6048091B604833010F01092E9
:101B1000B60492959F709F5F9093B9048091B90429
:101B2000823018F482E08093B904F999FECF8DE0F9
:101B300090E092BD81BDF89A60B5862F8C59893CA2
:101B400008F42AC160ED72E183E190E0F8946093BB
:101B5000090270930A0280930B0290930C02F99988
:101B6000FECF8EE090E092BD81BDF89A40B549303D
:101B700008F409C142E08CE08093B3044093AC04C4
:101B80000E946D2E789400E010E01DC08091FC044E
:101B90000E9499170E94D618C801849668E270E0E6
:101BA0000E94364A0E946C1A0E94FF1680E10E9431
:101BB000A20FC80187709070892B69F00F5F1F4FCB
:101BC0000C32110579F0083208F7802F0E946C1A48
:101BD0000E94C716DBCF0E9415160F5F1F4F0C32F5
:101BE000110589F70E9476170E94D6180E941516D3
:101BF00080E00E945014882331F083E00E9450144A
:101C0000882309F022C183E00E945014882309F040
:101C1000D3C08091FC048093E606109227071092AF
:101C2000BA051092430681E08093490610924A0655
:101C30008091E6066091270740914306209149066E
:101C40000DE816E00E94712D60914306C8010E94C4
:101C5000AA2A0E94352A0E94151680914C0483609E
:101C600080934C0410924D048091F704873009F45E
:101C700087C08830B0F5823009F45EC0833008F048
:101C800045C0882309F452C0813009F452C00E9433
:101C9000151680915404882359F080915404815082
:101CA000809354040E94AE04809154048823A9F7C1
:101CB0000E94352A882379F68091F704863039F717
:101CC00081E00E947C14882311F380E00E9450146C
:101CD0008823E9F20E9476170E94D618E0E0F0EF20
:101CE00019948C3009F449C08D3038F4883069F18A
:101CF0008B3069F60E948A24AECF8E3019F18E3077
:101D0000F0F08F3021F60E940C2FA5CF843059F0CF
:101D1000843030F0853009F0BACF0E94B8359BCFBF
:101D20000E941F2798CF0E945F1E95CF0E94D3125A
:101D300092CF0E9431428FCF0E9412408CCF0E94DE
:101D4000C34889CF0E94BF1A86CF0E9476170E948F
:101D5000151680915404882359F0809154048150C1
:101D6000809354040E94AE04809154048823A9F700
:101D70000E94352A882359F36ECF0E944D116BCFF4
:101D80000E948C2868CF242F30E0C901880F991F4A
:101D9000820F931F880FF0CE772767FD7095872FEE
:101DA000972F22EE34E040E050E00E94F749605364
:101DB0007D4E8C4E9F4FCACE8CE00E9450148823DB
:101DC00009F427CF6E010894C11CD11CFF24B1E196
:101DD000AB2EB12CAC0EBD1EAFE0EA2E86010E94E8
:101DE0001B01F801908381830E5F1F4F0A151B05AD
:101DF000B1F7F60104C03196E017F10789F02081B0
:101E0000822F90E08F7090700D9724F0822F8F704A
:101E10008083282F2D3079F78E2F8C198F3099F4ED
:101E200080E060E04F2D21E086010E94E62D85E5EF
:101E30000E948B1A0E94D618F394F0E8FF1671F6F0
:101E40000E947617E6CEE082D6CF1092440410921C
:101E500086046091860470E061707070629572957E
:101E6000707F7627607F762782E090E00E948B0269
:101E70000E946D2E1092CF041092BC0483E090E07B
:101E800060E00E948B0284E090E06091BC040E94BC
:101E90008B0288E790E0909399048093980485E002
:101EA00090E068E770E00E94950280E18093000274
:101EB0006091000287E090E00E948B021092B604CD
:101EC00088E08093B9048091B9046091B60490E0F1
:101ED000019782959295907F9827807F9827682B0D
:101EE0008AE090E00E948B028DE090E060E00E942A
:101EF0008B02F89480ED92E1A3E1B0E080930902B7
:101F000090930A02A0930B02B0930C0278948CE099
:101F10008093B30482E08093AC048EE090E062E0B2
:101F20000E948B0210E082E20E94331783E20E943B
:101F300033170E94D61882E30E94A20F1F5F183247
:101F400091F77ECF20EA3FE0E22FF32F3197F1F7B0
:101F50008A95D1F70895882309F41EC09AEF20EAE4
:101F60003FE0E22FF32F3197F1F79A95D1F7E22F67
:101F7000F32F3197F1F79A95D1F7E22FF32F31979D
:101F8000F1F79A95D1F7E22FF32F3197F1F79A9560
:101F9000D1F7815009F0E5CF08951092C504109251
:101FA000CE0408951F93CF93DF93EC01142F6F7726
:101FB0007885772309F44CC0462F50E0888190E063
:101FC0008F7790704817590779F121E030E00DC004
:101FD000D901FE01E20FF31F808190E08F779070AE
:101FE0002F5F3F4F8417950709F1271788F3272F95
:101FF0002F5F293030F128E0922F822F9150FE017F
:10200000E80FF11DDE01A90FB11D8C918083892F8E
:102010009923A1F71536C0F480E0862B88832887A2
:10202000DF91CF911F910895A0E0B0E0153670F4D4
:1020300080E0AC0FBD1F862B8C93DF91CF911F9159
:1020400008952223C9F6E6CF80E8E7CF80E8F1CFF4
:1020500091E081E021E0D2CFCF93DF93EC0138858E
:102060003323B9F06F7770E0888190E08F779070BC
:102070006817790789F0FE0120E008C0818190E0AF
:102080008F77907031966817790739F02F5F231793
:10209000A8F3DF91CF91089520E0323068F0922FBD
:1020A0009F5FFE01E20FF11DDE01A90FB11D8C91B2
:1020B0008083292F9317A0F331503887DF91CF9178
:1020C0000895282F9091BC048091C00085FFFCCF1B
:1020D00090699093C6008091C00085FFFCCF822F4D
:1020E0008F778093C60027FD09C0909137028091B9
:1020F000C00085FFFCCF9093C600089590913502F3
:102100008091C00085FFFCCF9093C6000895282FD2
:102110009091BC048091C00085FFFCCF90689093A3
:10212000C6008091C00085FFFCCF822F8F778093FF
:10213000C60027FD09C0909137028091C00085FF3D
:10214000FCCF9093C6000895909135028091C00015
:1021500085FFFCCF9093C6000895982F8091C00012
:1021600085FFFCCF9093C60080E090E008959091A9
:102170005F048091600420E030E0981711F021E0C6
:1021800030E0C901089590915F0480916004981730
:10219000D1F3F89490915F04E92FF0E0E053FB4F06
:1021A00080819F5F90935F0490915F049F719093F3
:1021B0005F04789490E0089590915F0480916004AA
:1021C000981729F00E94C310482F87FD03C040E0F4
:1021D000842F0895582F52955F705F30C9F3282FD0
:1021E00030E02F7030708091CF0490E028173907CD
:1021F00071F750935C04ECCF9091BC048091C000C7
:1022000085FFFCCF906B9093C6008091C00085FF46
:10221000FCCF8BE78093C6008091C00085FFFCCF88
:102220001092C600089580914404823049F0809154
:10223000C00085FFFCCF8CEF8093C6000E94FC108D
:102240000895909146048913089580E00E94571ED6
:102250008FEF8093460408951F93182F962F6623BF
:10226000B9F060E0809146048F3F09F061E0953657
:1022700048F4812F895140E00E94401E109346048B
:102280001F910895812F895141E00E94401EF6CF91
:1022900060E00E9421111F910895FF920F931F93F8
:1022A0008091A70581708093A7058091A7058093F1
:1022B0008E040E9476178091A705882309F032C109
:1022C0000E94D6188BE090E00E948402809338022E
:1022D0008CE090E00E94840280933902FF2410E099
:1022E0000E9415160E94E20C0E94352A882309F0EC
:1022F0004AC090915F0480916004981769F00E9431
:10230000C310682F87FD6DC080915C04883009F48C
:10231000AEC0893009F479C0112371F42091C5044D
:10232000222349F48091CE04882329F48091340734
:10233000882309F4E2C010E087E10E94A5148823F5
:1023400079F28091A7058F5F8093A7058091A705FB
:1023500081708093A7058091A70580938E0480E00B
:102360000E94FF168091A705882309F4B9CF80E069
:102370000E94C7160E9415160E94E20C0E94352A80
:10238000882309F4B6CF0E94FC1081E080934906AF
:10239000809127078093BA0510924A068091E6063D
:1023A0006091270740914306209149060DE816E009
:1023B0000E94712D60914306C8010E94AA2AFF2045
:1023C00061F08BE090E0609138020E948B028CE01B
:1023D00090E0609139020E948B021F910F91FF9053
:1023E0000895482F42954F704F3009F498C0282F18
:1023F00030E02F7030708091CF0490E028173907BB
:1024000009F48DC010925C046BCF67FDBAC0062F33
:102410000E94C310482F112309F08ECF509138022B
:10242000051748F0852F90E00F96202F30E0821797
:1024300093070CF082C050913902051708F46ECF53
:10244000852F90E00C96202F30E0821793070CF434
:1024500065CF051B86EC94E0602F0E94D20F80911F
:10246000C6048F778093D5062091C50459CF67FDA8
:1024700084C0062F0E94C310112371F540913802C9
:10248000041748F0842F90E00F96202F30E0821739
:1024900093070CF06BC040913902041708F43ECF4B
:1024A000842F90E00C96202F30E0821793070CF4D5
:1024B00035CF041B86EC94E0602F0E942C10809195
:1024C000CE04882309F42ACF8091C6048F778093A5
:1024D000D5062091C50424CF113009F456C089E1F6
:1024E0000E94FF16009339028091A70580938E0405
:1024F0002091C504FF24F39413CF84E00E94A51417
:102500008823A1F485E00E94A514882309F413CF41
:1025100010928E0489E10E94C71612E00DCF4093FD
:102520005C04F2CE80E00E94C716CACE10928E04E0
:1025300080E20E94C71611E0FFCE051B8DEB94E0F0
:10254000602F0E94D20F2091C50420935D048091DA
:10255000BD048F7780935E048091FC0490915E04AB
:102560008295807F890F80935E04DACE041B8DEB09
:1025700094E0602F0E942C10E6CF0E94C310082F19
:1025800079CF0E94C310082F43CF80E20E94FF162C
:10259000009338028091A70580938E042091C50492
:1025A000FF24F394BDCE1F930E948B178091CF041C
:1025B0000E9499170E94151684E60E94A20F0E949D
:1025C000151684E60E94A20F0E9415168FEF8093C5
:1025D00046040E9415160E94E20C0E94352A8823A8
:1025E00011F590915F0480916004981791F30E9417
:1025F000C310482F87FD1BC080915C04883049F1CF
:10260000893039F747FD32C0142F0E94C310682F5C
:10261000812F0E942C110E9415160E94E20C0E942C
:10262000352A8823F1F20E94FC101F910895582F3B
:1026300052955F705F30B9F0282F30E02F70307006
:102640008091CF0490E02817390769F010925C045C
:10265000C0CF47FD0FC0142F0E94C310682F812FD9
:102660000E942111B6CF50935C04C6CF0E94C310C4
:10267000182FCBCF0E94C310182FEECF1F920F92AE
:102680000FB60F920BB60F9211242F933F934F93D7
:102690005F936F937F938F939F93AF93BF93EF93CA
:1026A000FF939091C6009A3F09F442C09C3FA9F164
:1026B000983F09F44AC080916004E82FF0E0E053AD
:1026C000FB4F90838F5F80936004809160048F71D3
:1026D000809360049091600480915F04981751F496
:1026E00080915F048F5F80935F0480915F048F719E
:1026F00080935F04FF91EF91BF91AF919F918F9174
:102700007F916F915F914F913F912F910F900BBEF1
:102710000F900FBE0F901F90189580918E04882304
:1027200049F380914404823029F70E94CB2EE2CFF6
:10273000809144048230F1F680918E04882311F058
:102740000E94CF330E948900D5CF8091930490914D
:102750009404909343048093420410929404109242
:10276000930480914404823029F680916204909110
:102770006304892B31F05C98809154048F5F8093BF
:1027800054048091420490914304969587959093C8
:10279000630480936204809154048F5F8093540497
:1027A000A9CF80914404813009F05F98089599B1D0
:1027B000991F9927991F80916404882311F4992304
:1027C00021F49093640480E008959093640481E080
:1027D000089599B1991F9927991F809165048823BD
:1027E00011F0992321F09093650480E008951092F0
:1027F000650481E008958AB1806F8AB98BB18F70CA
:102800008BB908958AB18F708AB98BB18F708BB9EB
:10281000089580914404882321F45C9881E00E940B
:10282000A20F5F9A0895AC01F89428980000000068
:1028300000000000289A20E030E01EBC0DB407FE26
:10284000FDCF8EB5FA01E20FF31F80832F5F3F4F5C
:102850002330310591F77894089516980895169AC3
:10286000089520B1269526952F70822F90E0269509
:10287000322F369536952270322B880F991F282FCC
:102880002470322B880F991F880F991F8870382B5E
:102890008FE0831B089580B1869586958F7008958B
:1028A000282F883188F4E82FE695E695E695F0E044
:1028B000E350FB4F808190E0277002C0959587958B
:1028C0002A95E2F78170089580E00895282F8831D5
:1028D00088F4E82FE695E695E695F0E0EC50FB4F9E
:1028E000808190E0277002C0959587952A95E2F740
:1028F0008170089580E00895282F883188F4E82FAA
:10290000E695E695E695F0E0E850FB4F808190E093
:10291000277002C0959587952A95E2F781700895F2
:1029200080E008958091FD04882321F48091FE04C5
:10293000882319F090E0892F089590E08091FF049A
:102940008823C9F791E0892F0895282F8831A0F4B2
:10295000482F469546954695277081E090E0382FA0
:1029600001C0330F2A95EAF7A42FB0E0FD01EC5027
:10297000FB4F8081832319F420E0822F0895232FB9
:1029800030E020953095A350BB4F8C9190E02823E8
:102990003923232B89F7342F3F5F832F63E00E9475
:1029A000164AE92FF0E0E350FB4F8081882321F79E
:1029B00020E0832F8F5F0E94164AE92FF0E0E3505A
:1029C000FB4F80818823C9F621E0D7CF1F93CF9397
:1029D000DF93CCE4D2E010E088810E945014882379
:1029E00029F41F5F21961D30B9F71FEF812FDF916A
:1029F000CF911F9108951F93CF93DF93CCE4D2E042
:102A000010E088810E946614882349F41F5F219694
:102A10001D30B9F780E0DF91CF911F910895812F8C
:102A20008F5FDF91CF911F9108951F93CF93DF9315
:102A3000CCE4D2E010E088810E947C14882349F421
:102A40001F5F21961D30B9F780E0DF91CF911F9174
:102A50000895812F8F5FDF91CF911F9108951F936C
:102A6000CF93DF93C4E4D2E010E088810E94501439
:102A7000882349F41F5F21961830B9F780E0DF9171
:102A8000CF911F910895812F8F5FDF91CF911F917B
:102A900008951F93CF93DF93C4E4D2E010E08881C0
:102AA0000E946614882349F41F5F21961830B9F7F5
:102AB00080E0DF91CF911F910895812F8F5FDF918B
:102AC000CF911F9108951F93CF93DF93C4E4D2E079
:102AD00010E088810E947C14882349F41F5F2196AE
:102AE0001830B9F780E0DF91CF911F910895812FC1
:102AF0008F5FDF91CF911F910895CF93DF93C4E44F
:102B0000D2E088810E945014882349F4219682E003
:102B1000CC34D807B1F780E0DF91CF91089581E000
:102B2000DF91CF910895FF920F931F93CF93DF937F
:102B3000C4E4D2E0FF2400E006C00F5F219682E0EB
:102B4000CC34D80789F01881812F0E945014882333
:102B5000A1F7812F0E947C14882381F3F39421969E
:102B600082E0CC34D80779F781E0F81639F080E0BC
:102B7000DF91CF911F910F91FF90089580E0073072
:102B8000B9F781E0F5CF1F93CF93DF93CAE3D2E08B
:102B900010E088810E946614882349F41F5F219603
:102BA0001A30B9F780E0DF91CF911F910895812FFE
:102BB0008F5FDF91CF911F910895809167041092EC
:102BC0006704089580E00895382F883100F5282F94
:102BD000277081E090E0982F01C0990F2A95EAF7BD
:102BE000832F869586958695A82FB0E0FD01EC5041
:102BF000FB4F8081892369F4FD01E850FB4F808100
:102C0000892371F4A350BB4F8C91982339F480E051
:102C10000895832F0E94A51982E0089583E0089506
:102C2000832F0E94AD1981E00895EF92FF920F93D8
:102C30001F93DF93CF9300D000D0CDB7DEB71092B3
:102C4000F4041092F8041092F5041092F904109212
:102C5000F6041092FA04809168048A3068F426968B
:102C60000FB6F894DEBF0FBECDBFCF91DF911F919D
:102C70000F91FF90EF9008951092680416987E01CE
:102C80000894E11CF11CC7010E9413148091FD04FB
:102C90008C838091FE048D838091FF048E8360E09D
:102CA00070E001E010E0E62FE695E695E695F0E0AD
:102CB000CB0187709070980102C0220F331F8A9554
:102CC000E2F7C901AF0143505B4FD701AE0FBF1F01
:102CD0003C91E050FB4F2081232B28238095FA0163
:102CE00030818323282B20836F5F7F4F68317105EC
:102CF000D1F60E943114982F96959093FC048093FE
:102D0000F204169A40E050E0BE016C5F7F4FDA019A
:102D1000A050BB4FF701E40FF51F80818C93FB019E
:102D2000E40FF51F2081FA01E350FB4F9081FA0177
:102D3000EC50FB4F822F809589238083FA01E85065
:102D4000FB4F9095922390834F5F5F4F4330510527
:102D5000F1F690B1969596959F708091F004891741
:102D600021F0109269049093F004809169048F36E9
:102D700030F09093F1048091F1048093F00482E0AC
:102D80000E945014809353040E94D61868CF282FB5
:102D90008832C0F4E82FE695E695E695F0E02770D6
:102DA00081E090E001C0880F2A95EAF7DF01A6597B
:102DB000BB4F2C91282B2C93E159FB4F8095208100
:102DC000822380830895282F8832C0F4E82FE69567
:102DD000E695E695F0E0277081E090E001C0880F6D
:102DE0002A95EAF7DF01A159BB4F2C91282B2C9390
:102DF000E659FB4F80952081822380830895282FF8
:102E00008832C8F4E82FE695E695E695F0E027705D
:102E100081E090E002C0880F991F2A95E2F7809523
:102E2000DF01A659BB4F2C9128232C93E159FB4F6E
:102E30002081822380830895282F883298F4E82FF8
:102E4000E695E695E695F0E0E159FB4F277081E0C5
:102E500090E002C0880F991F2A95E2F780952081A3
:102E6000822380830895282F883290F4E82FE695F6
:102E7000E695E695F0E0E659FB4F277081E090E09B
:102E800002C0880F991F2A95E2F720812827208306
:102E90000895E82F883298F4282F277081E090E079
:102EA00002C0880F991F2A95E2F7E695E695E69508
:102EB000F0E0E159FB4F20812823822F089520E084
:102EC000822F0895982F969596959695EAE6F4E0C8
:102ED000E90FF11D208130E0877002C035952795FC
:102EE0008A95E2F721703070C901089510926E043E
:102EF00010926D0410926C0410926B0410926A048C
:102F00001092730410927204109271041092700463
:102F100010926F040895CF93DF93CAEBD2E08991AA
:102F20000E94FF1682E0CA3CD807C9F7DF91CF9113
:102F30000895803108F00895E82FF0E0E654FD4F41
:102F400080810E94C7160895803108F00895E82F07
:102F5000F0E0E654FD4F80810E94FF1608950F9324
:102F60001F93CF93DF93082FCAEBD2E010E007C086
:102F700088810E94C7161F5F2196103149F01017F3
:102F8000B8F388810E94FF161F5F21961031B9F7B0
:102F9000DF91CF911F910F910895803108F008952E
:102FA000E82FF0E0E654FD4F80810E94E31608957B
:102FB000803110F080E00895E82FF0E0E654FD4FF6
:102FC00080810E9462170895803110F080E008959A
:102FD000E82FF0E0E654FD4F80810E9449170895E4
:102FE000883108F00895E82FF0E0EB56FD4F80811E
:102FF0000E94C7160895883108F00895E82FF0E080
:10300000EB56FD4F80810E94E3160895883108F049
:103010000895E82FF0E0EB56FD4F80810E94FF16E7
:103020000895CF93DF93C5E9D2E089910E94FF16FE
:1030300082E0CD3AD807C9F7DF91CF910895E82F04
:103040008150883008F00895F0E0E457FD4F80810A
:103050000E94C71608950F931F93CF93DF93082FF5
:10306000CDE8D2E011E007C088810E94FF161F5F03
:103070002196193069F01017B9F7E12FF0E0E45705
:10308000FD4F80810E94C7161F5F2196193099F766
:10309000DF91CF911F910F910895E82F81508830D3
:1030A00008F00895F0E0E457FD4F80810E94FF167C
:1030B0000895E82F8150883008F00895F0E0E45733
:1030C000FD4F80810E94E3160895E82F81508830DB
:1030D00010F080E00895F0E0E457FD4F80810E94F9
:1030E00049170895E82F8150883010F080E0089546
:1030F000F0E0E457FD4F80810E9462170895CF935E
:10310000DF93CDE8D2E089910E94FF1682E0C539B5
:10311000D807C9F7DF91CF9108958D3008F0089551
:10312000E82FF0E0E355FD4F80810E94C716089517
:103130008D3008F00895E82FF0E0E355FD4F8081D1
:103140000E94FF1608958D3008F00895E82FF0E0F2
:10315000E355FD4F80810E94E3160895EDEAF2E009
:10316000E80FF11D80810E9449170895CF93DF93E6
:10317000CDEAD2E089910E94FF1682E0CA3BD807CF
:10318000C9F7DF91CF9108950E94B61884E00E949C
:10319000FF1683E00E94FF1688E00E94FF1681E080
:1031A0000E94FF1682E00E94FF160895F894179877
:1031B00020E030E090917404F901E159FB4F8081E7
:1031C0009823F901E659FB4F8081982B9EBD0DB4E1
:1031D00007FEFDCF2F5F3F4F2530310559F7179A76
:1031E00078940895EAE6F4E0AFE6B4E080819D913A
:1031F000892B819384E0EF36F807C1F70895EAE65A
:10320000F4E0AFE6B4E09D919095808189238193AD
:1032100084E0EF36F807B9F70895EAE6F4E0AFE6A0
:10322000B4E020819C91892F822319F090959223FC
:1032300090831D92319684E0EF36F80791F7089558
:103240001F93182F84E00E94FF16123049F083E08C
:103250000E94FF16113071F01F3F39F01F91089541
:1032600083E00E94E3161F91089584E00E94C71630
:103270001F91089583E00E94C7161F9108950F9330
:103280001F93CF93DF93182F87FD50C086E10E94D4
:103290000618812F829586958695837080FF29C0B8
:1032A00085E10E94F0171F7349F11731A0F58FEFE8
:1032B0000E94201984E10E940618012F10E0CBE043
:1032C000D0E0C017D10731F0FE01EE55FD4F8081EF
:1032D0000E94FF162196C831D10599F70E551D4F52
:1032E000F80180810E94C716DF91CF911F910F9145
:1032F000089585E10E9406181F73B9F680E00E94C8
:1033000020190E94B61884E10E94F017DF91CF9136
:103310001F910F910895143268F0103370F4185112
:1033200081E00E942019112329F6EBCF86E10E944B
:10333000F017AFCF1C5080E0F4CF1C3318F41452B8
:1033400082E0EFCF105383E0ECCFE5E9F2E0E80F45
:10335000F11D80810E94C7160895E5E9F2E0E80FAB
:10336000F11D80810E94FF160895EDE8F2E0E80F5C
:10337000F11D80810E94C7160895EDE8F2E0E80F84
:10338000F11D80810E94FF160895DF92EF92FF9257
:103390000F931F93CF93DF93F02EDE2C222371F136
:1033A000022F040FE42ECDE8D2E010E00BC010177E
:1033B00058F41F15D9F088810E94C7161F5F219607
:1033C000183049F01E1598F788810E94FF161F5F7C
:1033D00021961830B9F781E08D15A0F4DF91CF91D7
:1033E0001F910F91FF90EF90DF900895E12FF0E093
:1033F000E357FD4F80810E94E316E0CF062F080FB0
:10340000E82ED1CFDD2071F088E00E94FF1681E028
:103410000E94C716DF91CF911F910F91FF90EF90FF
:10342000DF90089588E00E94C71681E00E94FF1691
:10343000DF91CF911F910F91FF90EF90DF90089552
:10344000FF920F931F93082FF62E84E00E94FF1621
:1034500083E00E94FF1688E00E94FF1681E00E9430
:10346000FF16102F04FD34C015FD29C007FD2CC028
:1034700016FD21C00E94B618FF2099F0802F8F7092
:103480008D3098F08BE10E94C7168CE10E94C71620
:103490008FE00E94C7168EE00E94C7168DE00E9442
:1034A000C7161F910F91FF9008950E948D181F91CC
:1034B0000F91FF90089581E00E94C716DBCF83E053
:1034C0000E94C71607FFD4CF88E00E94C716D0CF4E
:1034D00084E00E94C716C8CFE9E5F2E0E80FF11DCD
:1034E000808108958C3008F00895E82FF0E0EF57C0
:1034F000FD4F80810E94C7160895CF93DF93C1E8E6
:10350000D2E089910E94FF1682E0CD38D807C9F732
:10351000DF91CF91089590916A04982790936A045F
:1035200090916B04982790936B0490916C0498276A
:1035300090936C0490916D04982790936D049091F2
:103540006E04982790936E040895AC01611571057F
:10355000A1F020E0E0E0A0E0B0E0A40FB51F8C9166
:10356000E827F0E0EE52FD4FE0812F5FA22FB0E0A0
:10357000A617B70790F38E2F0895E0E0FCCF0E94C6
:1035800015160E94E20C0E94352A8823C1F3089583
:10359000EF92FF920F931F93CF93DF937C018B01E8
:1035A0006115710561F0C0E0D0E0F701EC0FFD1F7F
:1035B00080810E9409022196C017D107B0F3DF91E4
:1035C000CF911F910F91FF90EF90089522E42093E7
:1035D00003051092040522E020930505909306054B
:1035E00080930705A3E0B5E0E0E08D91E827F0E0E7
:1035F000EE52FD4FE08185E0A830B807B1F7EC93BB
:10360000CD01059766E070E00E94C81A089590E821
:10361000909303051092040521E020930505809303
:103620000605A2EDB2E090915203FD01E90FF11DF4
:1036300090819227FD01E90FF11D90819827A90F34
:10364000B11D8C918093070583E095E065E070E003
:103650000E94C81A08951F920F920FB60F920BB6D0
:103660000F921124DF92EF92FF920F931F932F93EB
:103670003F934F935F936F937F938F939F93AF93FA
:10368000BF93CF93DF93EF93FF931091CE00809180
:10369000D102882309F46EC0809177049091780458
:1036A000895E934008F080C080917504803408F0F2
:1036B00089C0282F2F5FE82FF0E0ED5BFA4F1083D1
:1036C000209375041092780410927704233008F444
:1036D00051C0709143059091440580E0609145058B
:1036E000462F50E0482B592B30E0CA01049628178A
:1036F000390708F43FC09A012D5F3F4FF901ED5B98
:10370000FA4F10812115310509F401C190E0E0E084
:10371000A0E0B0E0AD5BBA4F8C91E827F0E0EE524C
:10372000FD4FE0819F5FA92FB0E0A217B30790F390
:103730001E1709F450C02115310509F4EAC090E0C4
:10374000E0E0A0E0B0E0AD5BBA4F8C91E827F0E09C
:10375000EE52FD4FE0819F5FA92FB0E0A217B307A3
:1037600090F38E2F90E00E94E5011092750480E0A6
:103770000E94071BFF91EF91DF91CF91BF91AF9115
:103780009F918F917F916F915F914F913F912F9179
:103790001F910F91FF90EF90DF900F900BBE0F9055
:1037A0000FBE0F901F9018950E948B170E94D6187D
:1037B0001093430581E08093750410927804109271
:1037C0007704D8CF0E94071B1092750410927804DA
:1037D00010927704CFCF713809F492C17238B0F5E6
:1037E000713109F42BC1723108F096C0713051F17A
:1037F000703131F080E00E94071B10927504BACF3F
:103800006231C1F780914605082F10E0000F111FAB
:10381000000F111F000F111F80914705080F111D88
:1038200002951295107F1027007F1027C8E4D5E07D
:103830008991B8010E94221F0F5F1F4F85E0C83594
:10384000D807B1F781E00E94071BD7CF763809F47B
:1038500035C1773808F073C0723809F484C17538FF
:1038600049F64330510509F0A5C030914605932F24
:1038700080E020914705E22EFF24E82AF92AD09023
:103880004805EAE3ED1508F4B6CF709303051092EE
:103890000405F2E0DF0ED09205058EEFD80E3093CE
:1038A000060520930705DD2071F008E015E0E7012B
:1038B000CE010E94661FF80181938F0121969E011F
:1038C0002E192D15A8F380910505682F6D5F09F459
:1038D000D5C1A3E0B5E090E08E5F282F30E02C5FEB
:1038E0003A4F8D919827E92FF0E0EE52FD4F9081ED
:1038F000A217B307B1F7E62FF0E0ED5FFA4F908320
:103900006F5F83E095E070E00E94C81A76CFE0E038
:103910000FCF80E090E027CF703409F453C17134A9
:1039200009F068CF623009F065CF9091460580E0DC
:1039300020914705820F911D0E94F1025ECF7738DA
:10394000E9F1783809F056CF709303051092040519
:1039500080914605813009F46AC1813008F05BC16D
:1039600080E1809306051092070580930805109268
:10397000090584E047E0A7E0B0E068E070E08093EC
:10398000050590E020E030E0F901ED5FFA4F80811D
:103990009827E92FF0E0EE52FD4F90812F5F3F4FC7
:1039A000241790F3AD5FBA4F9C9383E095E00E949B
:1039B000C81A23CF80E00E94071B1FCF80914605C5
:1039C000882309F006C14230510509F014CFE09177
:1039D0004705E43008F00ECF89E18093030510928B
:1039E000040580E1809305052E2F30E02295329565
:1039F000307F3227207F3227A6E0B5E0F901E35778
:103A0000F94F80818D932F5F3F4F85E0A631B80736
:103A1000A9F75397E0E08D91E827F0E0EE52FD4FD3
:103A2000E081F5E0A631BF07B1F7E0931605CD01BF
:103A3000439764E170E00E94C81ADFCE623009F05B
:103A4000D9CE80914605082F10E0000F111F000FFE
:103A5000111F000F111F80914705080F111D0295BE
:103A60001295107F1027007F102789E180930305AE
:103A70001092040580E180930505C6E0D5E0C801F9
:103A80000E94661F89930F5F1F4F35E0C631D30731
:103A9000B1F7DE015397E0E08D91E827F0E0EE52B8
:103AA000FD4FE081CA17DB07B9F7E093160583E005
:103AB00095E064E170E00E94C81A9FCE909146059F
:103AC00080E020914705E22EFF24E82AF92A2EEF14
:103AD000D22ED60E63506A3308F06CCFDD2009F485
:103AE000B1CE08E415E0E701F80181918F01BE0134
:103AF0000E94221F21969E012E192D15A8F3A2CEF9
:103B000087E190E090930705809306058FEC90E0A5
:103B10009093090580930805EAECF2E0AAE0B5E08D
:103B200081918D9322E0E03DF207D1F781E8809307
:103B30000305109204058AE080930505A3E0B5E033
:103B4000E0E08D91E827F0E0EE52FD4FE08135E0B6
:103B5000A031B307B1F7EC93CD010D976EE070E0A3
:103B60000E94C81A4ACE4230510509F023CF309145
:103B70004605332309F468C09091470520E082E8A8
:103B8000809303051092040583E08093050530932C
:103B900006059093070520930805A3E0B5E0E0E053
:103BA0008D91E827F0E0EE52FD4FE08185E0A930ED
:103BB000B807B1F7EC93CD01069767E070E00E947B
:103BC000C81A1BCE80919804909199040E94E61A1D
:103BD00014CE813009F00ECE4231510509F00ACEE3
:103BE000E0914705E43008F005CE2E2F30E0A8E440
:103BF000B5E022953295307F3227207F32278D9194
:103C0000F901E357F94F80832F5F3F4F85E0A835D7
:103C1000B807A9F717CE883009F0ECCD81E0809382
:103C2000060544E0A4E0B0E065E070E0A8CE88E0DE
:103C30008093060580E18093070582E045E0A5E0DA
:103C4000B0E066E070E09BCE90914705973860F455
:103C5000953870F4993181F0993120F0892F81588D
:103C6000823030F020E08BCF973821F09838D1F7B0
:103C700021E085CF24E083CF20E181CF90E03BCECF
:103C80002C98803408F08FE3611160E4442349F0FC
:103C900090E0882349F0682B962B98B92C9A2D9A9E
:103CA000089590E88823B9F7962B98B9089588234A
:103CB00019F42D982C980895469A2C9808959F925F
:103CC000AF92BF92CF92DF92EF92FF920F931F932A
:103CD000CF93DF930E948B178091BC040E949917A9
:103CE0000E9415160E94DD15BB249924AA24CC2419
:103CF0000E9415160E94E20C0E94352A882309F0C2
:103D000075C02B2D3CE02302C001112497E1D92E70
:103D1000D80EEA2CE294EE0CEE0C80ECE822C0E027
:103D2000D0E009C0802F0E947C14882319F52196C9
:103D3000CD30D10559F1FC2EFE01EE52FC4F008131
:103D4000802F0E946614882369F31C2F1D0D812F7C
:103D50006C2D4A2D0E94401E812F8E290E946110D9
:103D60008C2F0E948D18CC24C394802F0E947C1429
:103D70008823E9F28F2D8D0D8E290E9487108F2DBB
:103D80000E9498182196CD30D105A9F68FE00E94A7
:103D90006614882309F444C081E08B150CF050C0F0
:103DA0009B1429F08B2D0E9420190E94D61884E1C3
:103DB0000E946614882351F080E0AA2009F481E073
:103DC000A82E8823C9F188E00E94C71686B190E02A
:103DD0008F739070892BC1F49B2C0E9415160E9442
:103DE000E20C0E94352A882309F48BCF0E94FC1034
:103DF000DF91CF911F910F91FF90EF90DF90CF90C7
:103E0000BF90AF909F9008950E949214882321F351
:103E100080E00E94571E0E94B618CC249B2CDDCF58
:103E20008EE00E946614882309F4BACF2FEFB216F1
:103E300009F4B6CFBA94B4CF88E00E94FF16C6CF7B
:103E4000B394AECF282FF89495E028980000000096
:103E5000000000009EBD0DB407FEFDCF0000000075
:103E6000000000001EBC0DB407FEFDCF8EB5289AE1
:103E7000000000000000000080FDE7CF289800004F
:103E8000000086E08EBD0DB407FEFDCF00000000EF
:103E9000289A0000000000000000289800000000A0
:103EA00082E08EBD0DB407FEFDCF7EBD0DB407FED2
:103EB000FDCF6EBD0DB407FEFDCF2EBD0DB407FEC8
:103EC000FDCF00000000289A78940895382FF894C8
:103ED00025E0289800000000000000002EBD0DB471
:103EE00007FEFDCF00000000000000001EBC0DB466
:103EF00007FEFDCF8EB5289A0000000000000000EC
:103F000080FDE7CF28980000000083E08EBD0DB44F
:103F100007FEFDCF9EBD0DB407FEFDCF3EBD0DB427
:103F200007FEFDCF000000001EBC0DB407FEFDCF54
:103F30008EB5289A78940895892F8F7184FD806EAC
:103F40000895EF92FF920F931F93FA01D90186957E
:103F50008083862F90E08F709070959587959595CA
:103F60008795959587958C93862F8770F801808328
:103F700062956F70F70160831F910F91FF90EF9032
:103F80000895FC0130E022953295307F3227207F62
:103F9000322720838081660F660F660F640F6F7073
:103FA000862B8083089580917904882349F087FDCA
:103FB0000EC083E00E94C71684E00E94FF16089599
:103FC00083E00E94FF1684E00E94FF16089583E0BC
:103FD0000E94FF1684E00E94C7160895EF920F9387
:103FE0008091A3059091A40580E00E94A5148823E8
:103FF000A1F58091B705813009F448C080E00E94A6
:104000007C14882319F40F91EF90089582E20E94A6
:10401000C7161092B7052091B2053091B30521154E
:10402000310591F0E091B405F0E0EE0FFF1FE15291
:10403000FC4F808191818217930730F021503040EE
:104040003093A4052093A30580914E048230C1F1E2
:1040500010924E040F91EF90089581E08093B70580
:104060001092B3051092B20582E20E94FF16809171
:10407000A3059091A40501960E94260282E08093F8
:104080004E048091B705813009F0B8CF0E94C31566
:10409000482F882379F587E10E9466148823F9F474
:1040A00083E00E946614882309F4A8CF8091AE05AE
:1040B0009091AF050E94260282E080934E049ECF2D
:1040C00080914306609149064091BC0520914A06C3
:1040D00000914306E090BA050E94C519B9CF8091BE
:1040E000B5059091B60501960E94260282E0809364
:1040F0004E04D6CF41502091B2053091B305C9018D
:10410000880F991F880F991F880F991F220F331F3F
:10411000820F931F840F911D9093B3058093B20576
:104120000E94260282E080934E04B5CF962F803104
:1041300010F08FEF0895682F70E0660F771F6F5FA4
:10414000734F892F0E94221F80E008959B018031C8
:1041500020F5682F70E0FB01EE0FFF1FE152FC4FCE
:104160008081918128173907A0F0009749F081508C
:10417000660F771F6050744F0E94221F80E00895E1
:1041800080E0660F771F6050744F0E94221F80E00E
:104190000895C901009759F7F3CF8FEF0895803143
:1041A00098F470E06050784F90E0002496958795E1
:1041B0000794969587950794982F802D680F791FFF
:1041C0008CE06030780710F08FEF0895842F0E9404
:1041D000221F80E00895EF92FF920F931F93CF93D9
:1041E000DF93C82FD0E0CC0FDD1FCC0FDD1FCC0F2D
:1041F000DD1FC60FD11DC05CDF4FCC0FDD1FC29588
:10420000D295D07FDC27C07FDC27EE24FF248701F6
:10421000000F111F0D571A4FF80180819181892FCE
:10422000BE010E94221FF801808191812196BE016A
:104230000E94221F0894E11CF11C2196F0E1EF1668
:10424000F10429F7DF91CF911F910F91FF90EF902B
:10425000089590E0880F991F8F5F934F0E94661F0B
:1042600090E008950F931F93082F10E0000F111F87
:10427000C8018050944F0E94661F90E00196015241
:104280001C4FF801208131818217930708F49C01AB
:10429000C9011F910F9108958091F2048093B40594
:1042A0008091B4050E9432219093AF058093AE05B2
:1042B0008091B4050E9429219093B6058093B5059D
:1042C0002091B5053091B6058091AE059091AF056E
:1042D0002817390720F01092B6051092B505809185
:1042E000A3059091A405E091B405F0E0EE0FFF1F47
:1042F000E152FC4F608171810E94224A9093A40593
:104300008093A3050895803198F470E06050784F51
:1043100090E0002496958795079496958795079445
:10432000982F802D680F791F8CE06030780710F08F
:104330008FEF0895CB010E94661F0895CF92DF9200
:10434000EF92FF920F931F93DF93CF930F92CDB70E
:10435000DEB7C090A305D090A4050894C11CD11C61
:1043600080E00E94A5148823E9F419828091B705A2
:10437000813051F180E00E947C14882329F08091E3
:10438000B705882309F0C9C0E981E13009F4EEC01E
:104390000F90CF91DF911F910F91FF90EF90DF90E1
:1043A000CF90089581E08093B7051092B3051092E5
:1043B000B2058093800482E20E94FF1681E0898327
:1043C0008091B7058130B1F60E94C315282F88234C
:1043D000C1F021508091B2059091B3056C01CC0CD5
:1043E000DD1CCC0CDD1CCC0CDD1C880F991FC80E0D
:1043F000D91EC20ED11CD092B305C092B205E1E025
:10440000E98387E10E946614882349F0C090B505CE
:10441000D090B6050894C11CD11CF1E0F98383E06B
:104420000E946614882331F0C090AE05D090AF058D
:1044300081E0898389E00E946614882309F09DC089
:1044400089E00E947C14882309F0B5C08AE00E94AC
:104450006614882309F0A0C08AE00E947C14882397
:1044600009F488CF8CE10E94FF16E091B4052091F9
:10447000AE053091AF05F0E0EE0FFF1FE152FC4FAB
:10448000808191812817390708F074CF8091AE059B
:104490009091AF0501969093AF058093AE05809102
:1044A000B4056091AE057091AF050E94A620809181
:1044B000B4050E9432219093AF058093AE056091C0
:1044C000AE057091AF05615070408091A305909149
:1044D000A40586179707E8F47B010894E108F10822
:1044E00001C079018091B4051E2D6E2D0E9483219B
:1044F000482F8091B4051F5F612F0E94CF20970144
:10450000215030408091A3059091A4058E159F0500
:1045100040F388E0809383042DCF82E20E94C71687
:10452000109280041092B70581E08093830420915B
:10453000B2053091B3052115310569F0E091B4055C
:10454000F0E0EE0FFF1FE152FC4F80819181821756
:10455000930708F076C080914E04823009F47BC046
:1045600010924E04E981E13009F012CFC6010E9499
:10457000260282E080934E040BCF8BE10E94C71687
:104580001092B3051092B205C090A305D090A40577
:104590000894C11CD11C54CF8CE10E94C716109204
:1045A000B3051092B205C090A305D090A40508945D
:1045B000C11CD11C51CF8BE10E94FF16E090A305D6
:1045C000F090A4050894E11CF11C8091AE05909137
:1045D000AF05E816F90608F039CF8091B4051E2D15
:1045E0006E2D0E948321482F8091B4051150612FB8
:1045F0000E94CF200894E11CF11C8091AE0590919F
:10460000AF05E816F90648F38091AE059091AF0525
:1046100001979093AF058093AE058091B4056091AA
:10462000AE057091AF050E94A6208091B4050E944E
:1046300032219093AF058093AE0588E08093830488
:1046400005CF215030403093A4052093A30587E087
:104650008093830480CF8091430660914906409106
:10466000BC0520914A0600914306E090BA050E94DD
:10467000C51976CFEF92FF920F931F938091F204AA
:104680008093B4058091B4050E9432219093AF05C8
:104690008093AE058091B4050E9429219093B605C0
:1046A0008093B5052091B5053091B6058091AE0592
:1046B0009091AF052817390720F01092B605109297
:1046C000B5058091A3059091A405E091B405F0E0B3
:1046D000EE0FFF1FE152FC4F608171810E94224A60
:1046E0009093A4058093A3058091B4056091A305E0
:1046F0007091A4050E9483218093AB058091B4053D
:104700006091AB0542E056E02AEB35E00CEB15E09A
:104710009EECE92E96E0F92E0E94A11F81E0809385
:104720004A060E94662A8091CE068093D5061F9184
:104730000F91FF90EF900895AF92BF92CF92DF92CA
:10474000EF92FF920F931F93CF93DF93C82EDD2438
:10475000CC0CDD1CCC0CDD1CCC0CDD1CC60ED11C25
:1047600080E490E0C80ED91ECC0CDD1CC294D2941B
:1047700040EFD422DC24C422DC24AA24BB24C601BA
:104780000E94661FD82FC0E07501EE0CFF1CE3E805
:10479000F5E0EE0EFF1EF701D183C0830081118189
:1047A000C60101960E94661F90E0082B192BF701A5
:1047B000118300830894A11CB11C82E090E0C80E14
:1047C000D91E90E1A916B104D1F6DF91CF911F91C6
:1047D0000F91FF90EF90DF90CF90BF90AF90089532
:1047E0001092AD0584E20E94FF160E9476170E9487
:1047F0000D191092480680E00E94571E08951092ED
:10480000AC05109248061092A50580E00E94571E44
:104810000E9476170E940D190E94DD15089580915F
:10482000A9059091AA05682F67709695879596952A
:104830008795969587958F700E94352E6091A90572
:104840007091AA059B0140E050E0DA01C901807037
:104850009078A070B070892F9A2FAB2FBB278093D0
:104860008A04DA01C90180709074A070B070892F39
:104870009A2FAB2FBB278093880420703072407032
:104880005070232F342F452F5527209389041092E1
:10489000BD05872F8F7184FD806E089581E0809320
:1048A000AC0581E20E94C7161092880480918804AA
:1048B000809389048091890480938A041092A505CD
:1048C0001092480680918305909184059093AA05E3
:1048D0008093A9058F5F9F4F89F01092B1051092C8
:1048E000BD05109296040E940F2480937904809154
:1048F000450480FDFCCF81E08093A5050E948B17C5
:10490000089581E08093AD0584E20E94C7160E945D
:104910008B170895DF92EF92FF920F931F93809170
:104920003407882309F487C284E00E94EA2A10929F
:10493000A8058091A8058093A7051092B70510924D
:10494000B3051092B2050E943A238091E606609169
:10495000270740914306209149060DE816E00E9482
:10496000712D80914306609149064091BC052091CC
:104970004A060091C005E090BA050E94C51917E0EB
:10498000D12E07C0113009F4FFC00E94082D8823E2
:10499000D9F00E9415160E94E20C1091CD0613303A
:1049A000E9F0143078F31430E9F11D3071F781E04B
:1049B0000E941C348091CD068D3039F310928E0404
:1049C0000E94082D882329F70E94D72C0E941516D3
:1049D0000E94E20C1091CD06133019F70E94F02AC4
:1049E000882309F09EC10E94622C882321F0109236
:1049F000800410928E040E94FB14882331F2182F39
:104A000011500E94B618812F0E948D181093CE0667
:104A100080913407882309F0B8CF8091CE06809327
:104A2000D506B3CF0E94F02A882309F05CC180919B
:104A3000B705882309F44AC10E949E2183E00E94A1
:104A4000A514882309F03BC187E10E94A51488239F
:104A500009F02EC186E10E94A514882309F468C0DC
:104A600080914A06882309F0B0C18091CE068093D8
:104A7000D506E090A305F090A4058091A8058823B1
:104A800009F090C180914906882309F44AC010E0DA
:104A900020912707309143068091D50690E08295BA
:104AA0009295907F9827807F98278093AB0580917F
:104AB000AB05220F220F220F230F210F2F70282B5F
:104AC0002093AB058091B4056091A3057091A40576
:104AD0004091AB050E94CF201F5F8091A30590916C
:104AE000A40501969093A4058093A3050894E11C66
:104AF000F11C8091A3059091A405E091B405F0E02C
:104B0000EE0FFF1FE152FC4F608171810E94224A2B
:104B10009093A4058093A30580914906181708F483
:104B2000B7CF8091A705882309F052C1D0928304A2
:104B300080918304873009F407C180918304883011
:104B400009F459C180918304813009F4AEC0809189
:104B5000CD06843011F010928E04809134078823A2
:104B600009F4DBC080918D04813009F00ECF1092E2
:104B70008D040E94352A882309F407CF1F910F91D5
:104B8000FF90EF90DF9008950E94F02A882309F0AB
:104B900073C00E949E2183E00E94A514882339F5EA
:104BA00083E00E947C148823F1F49091B4058091F5
:104BB000F204981711F00E943A238091CD068130BB
:104BC00011F010928E0480913407882309F0B8C048
:104BD0000E94352A882309F4D8CE1F910F91FF90A7
:104BE000EF90DF90089583E20E94FF16DECF1092CF
:104BF000A4051092A3058091B4056091A30570915E
:104C0000A4050E9483218093AB058091B405609137
:104C1000AB0542E056E02AEB35E00CEB15E0BEECCC
:104C2000EB2EB6E0FB2E0E94A11F81E080934A0686
:104C30008091CE068093D5060E94662A8091E60672
:104C40006091270740914306209149060DE816E040
:104C50000E94712D80914306609149064091BC05E8
:104C600020914A060091C005E090BA050E94C5193E
:104C700083E20E94C71694CF0E94761782E20E94B8
:104C8000C71610938E0481E20E94FF16809143069E
:104C9000609149064091BC0520914A060091430667
:104CA000E090BA050E94C51974CF109283044FCFCB
:104CB00081E08093A80580E00E94E316CBCE81E0DE
:104CC0008093A70583E20E94E316BECE0E94F52CD6
:104CD0009091B40596959093FC04882309F0ACCE8E
:104CE0000E941C34A9CE0E94761782E20E94C71649
:104CF00081E080938E0481E20E94C7168091430672
:104D0000609149064091BC0520914A0600914306F6
:104D1000E090BA050E94C5198ACE81E00E94EA2A75
:104D200021CF0E94761711E01093800484E20E9444
:104D3000C7168091CE060E948D1810938E0453CE14
:104D400084E00E94EA2A44CF8091B4056091A305D3
:104D50007091A4050E9483218093AB058091B405D6
:104D60006091AB0542E056E02AEB35E00CEB15E034
:104D70007EECE72E76E0F72E0E94A11F11E0109343
:104D80004A0680914306609149064091BC052091F6
:104D90004A060091C005E090BA050E94C51910931B
:104DA0008304D0CE1092A8058091B4056E2D0E9488
:104DB00096208091B4050E9429219093B605809396
:104DC000B50580E00E94FF165DCE0E94662A4DCE9A
:104DD0001092A7058091B405B7010E94A62080918A
:104DE000B4050E9432219093AF058093AE0583E213
:104DF0000E94FF169BCE8091B4056091A30570912F
:104E0000A4050E9483218093AB058091B405609135
:104E1000AB0542E056E02AEB35E00CEB15E09EECEA
:104E2000E92E96E0F92E0E94A11F81E080934A06A8
:104E30001092830487CE81E00E94EA2A78CDEF9217
:104E4000FF920F931F9380913407882309F460C168
:104E500084E00E94EA2A1092A8058091A805809318
:104E6000A7051092B7051092B3051092B2050E94E3
:104E70003A238091E60660912707409143062091EE
:104E800049060DE816E00E94712D8091430660915D
:104E900049064091BC0520914A060091C005E0906A
:104EA000BA050E94C51908C0143009F456C00E9402
:104EB000082D882309F47DC00E9415160E94E20C7B
:104EC0001091CD06113081F70E94F02A882309F055
:104ED00087C083E00E94A514882309F0A2C083E064
:104EE0000E947C14882309F0E6C00E94EE1F909176
:104EF000B4058091F2049817E1F00E943A23809162
:104F0000E6066091270740914306209149060DE887
:104F100016E00E94712D80914306609149064091F0
:104F2000BC0520914A060091C005E090BA050E9498
:104F3000C5198091CD06813011F010928E048091B8
:104F400034078823C9F50E94352A882309F4AFCF96
:104F50001F910F91FF90EF9008950E94F02A8823EF
:104F600009F0B9C086E10E94A514882309F0A7C002
:104F700083E00E94A514882339F50E94EE1F8091DA
:104F8000CD06843011F010928E048091340788236E
:104F9000B9F080918D04813009F089CF10928D0491
:104FA0000E94352A8823A1F60E94082D882309F043
:104FB00083CF0E94D72C80CF84E00E94EA2AC3CFFF
:104FC00081E00E94EA2AE5CF81E08093A70583E291
:104FD0000E94C7161092A80580E00E94FF16CDCF50
:104FE0000E94761782E20E94C71610938E0481E217
:104FF0000E94FF1680914306609149064091BC05CE
:1050000020914A0600914306E090BA050E94C51916
:1050100081E00E94620283E00E94A514882309F4C3
:105020005ECF1092A4051092A3058091B405609103
:10503000A3057091A4050E9483218093AB05809104
:10504000B4056091AB0542E056E02AEB35E00CEB8D
:1050500015E09EECE92E96E0F92E0E94A11F81E05A
:1050600080934A068091CE068093D5060E94662AD8
:105070008091E606609127074091430620914906FA
:105080000DE816E00E94712D80914306609149065B
:105090004091BC0520914A060091C005E090BA05F8
:1050A0000E94C51983E20E94C71683E00E947C1407
:1050B000882309F41ACF83E20E94FF1616CF81E0FD
:1050C0008093A80580E00E94C7161092A70583E28E
:1050D0000E94FF164DCF0E94761782E20E94C716EB
:1050E00081E080938E0481E20E94C716809143067E
:1050F000609149064091BC0520914A060091430603
:10510000E090BA050E94C51981E00E9462022ACF90
:1051100081E00E94EA2A9FCEEF92FF920F931F93A5
:1051200010927B0480913407882309F49AC184E0AB
:105130000E94EA2A1092A8058091A8058093A705ED
:105140001092B7051092B3051092B2050E944C213F
:1051500022E0F22E07C0113009F494C00E94082DFD
:105160008823D9F00E9415160E94E20C1091CD06FA
:105170001330E9F0143078F31430E9F11D3071F791
:1051800081E00E941C348091CD068D3039F310925D
:105190008E040E94082D882329F70E94D72C0E9494
:1051A00015160E94E20C1091CD06133019F70E94DB
:1051B000F02A882309F0E8C00E94622C882321F09D
:1051C0001092800410928E040E94FB14882331F206
:1051D000182F11500E94B618812F0E948D1810931D
:1051E000CE0680913407882309F0B8CF8091CE068F
:1051F0008093D506B3CF0E94F02A882309F0EDC032
:105200008091B705882309F4DBC083E00E94A514D0
:10521000882329F080917B04813009F40DC187E156
:105220000E94A514882309F0C4C080E00E94A51440
:10523000882309F0A0C080E00E947C14882309F034
:105240008DC08091CD06843011F010928E04809133
:105250003407882309F4A7C080918D04813009F0B8
:105260007DCF10928D0480917B04882309F076CF46
:105270000E94352A882309F471CF1F910F91FF9066
:10528000EF9008950E94F02A8823B1F58091B70528
:10529000882309F456C083E00E94A514882379F07E
:1052A00081E080937B0480917B04882309F4B8C05B
:1052B00083E20E94C7161092A4051092A3050E94D3
:1052C000EE1F9091B4058091F204981711F00E949E
:1052D0004C218091CD06813011F010928E04809186
:1052E0003407882329F284E00E94EA2A0E94352AA2
:1052F000882309F433CFC1CF0E94761782E20E943F
:10530000C71610938E0481E20E94FF168091430617
:10531000609149064091BC0520914A0600914306E0
:10532000E090BA050E94C51980917B04882309F496
:105330007BC083E20E94C7168091B705882309F0DD
:10534000AACF0E94F52C9091B40596959093FC04F9
:10535000882309F0A0CF0E941C349DCF82E20E94D6
:10536000C7161092B70580914E04823009F46AC0C6
:1053700010924E0466CF81E08093B70582E20E94CE
:10538000FF16F0924E0457CF0E94761711E010934B
:10539000800484E20E94C7168091CE060E948D1878
:1053A00010938E0409CF81E00E94EA2A10927B04B8
:1053B00053CF81E08093A80580E00E94E31635CFAB
:1053C0000E94F52C9091B40596959093FC04882347
:1053D00009F01BCF0E941C3418CF0E94761782E27E
:1053E0000E94C71681E080938E0481E20E94C71656
:1053F00080914306609149064091BC0520914A0680
:1054000000914306E090BA050E94C51980917B0483
:10541000882371F083E20E94E3160E94D618F0CE32
:1054200083E20E94FF1647CF83E20E94FF162ECF31
:1054300083E20E94FF16F1CF8093A70583E20E94CA
:10544000C716EDCE80914306609149064091BC0598
:1054500020914A0600914306E090BA050E94C519C2
:1054600087CF81E00E94EA2A65CE9091F104809175
:10547000F704891731F08091F1048093F70481E0FB
:10548000089580E0089580914A06882391F08091E4
:1054900002068093E6068091BA05809327078091E3
:1054A000BC058093430680914A068093490610927A
:1054B0004A0680914906882329F080914906809305
:1054C0004906089581E08093490608958091020677
:1054D0008093E6068091BA05809327078091BC05EA
:1054E0008093430680914A068093490610924A06AB
:1054F0000895833059F0843050F0843029F0809141
:10550000CE068093D50608951092CE060895823077
:10551000B0F70895FC0187858F708D30C1F030E0C1
:1055200020E190E080818F708E3061F09F5F319636
:105530009217C0F3892F913118F48150832B08956D
:1055400080E1FBCF9923B1F780E0832B089530E110
:105550002FE0E7CF1F93DF93CF930F92CDB7DEB746
:10556000162F0E948A2A898389818F708F5F80938A
:1055700000041093C005898184FD08C08CE08093ED
:10558000FF030F90CF91DF911F91089580E18093E9
:10559000FF030F90CF91DF911F910895E82FF0E066
:1055A000EF73F070EE5FFB4F808108954093BE056E
:1055B000609301068093CD0681E0809346060895AE
:1055C000882339F0809101068093CD0681E0809395
:1055D000460608958093CD0681E08093460608959F
:1055E00080914606882319F01092460681E00895BE
:1055F0003F924F925F926F927F928F929F92AF9263
:10560000BF92CF92DF92EF92FF920F931F93CF93AF
:10561000DF93462E4A015901662309F4C4C09C0158
:10562000E90100E0FF241FEFDD2466247724B2E0C7
:105630005B2E33243394CE010E948A2AF301EF5269
:10564000F94F8083C0802FE0C222C39440E050E035
:1056500012C01E251F7BF1F4F501E00FF11D308211
:10566000FF2009F070C0DD24D3940F5F4F5F5F4FC0
:105670001E2D4C1588F5642FFE01E40FF51FE08008
:105680002E2D30E0C9018F7090700F9709F455C02E
:10569000DD20F9F6F501E00FF11D5082EF2DF0E06D
:1056A000D401AE0FBF1FEC926295607FE55BF94FAE
:1056B0006083F3940024220F331F001C220F331F3A
:1056C000001C232F302DDD24D394D2220F5F4F5F97
:1056D0005F4F1E2D4C1578F20894611C711C60966A
:1056E000641408F4A8CF003408F061C08F2DF501D0
:1056F000E00FF11D10820F5F0034C8F39FE39F1588
:1057000050F09FEFEF2DF0E0E55BF94F9083F394BD
:105710002FE32F15B8F7DF91CF911F910F91FF90D5
:10572000EF90DF90CF90BF90AF909F908F907F9041
:105730006F905F904F903F900895F501E00FF11D3D
:105740001082DD2492CFEF2DF0E03197E80DF91DA6
:10575000E082FA94EF2DF0E0F394E55BF94FA0813D
:10576000AF70BA2FBF5F808182958F70682F70E015
:10577000CB018B0F911D40970CF0BA2F0024220F04
:10578000331F001C220F331F001C232F302DDD245C
:10579000D394D22262957295707F7627607F7627A8
:1057A000B62BB08362CF00E0FF2480E0A0CF8F2D26
:1057B000A5CF2F923F924F925F926F927F928F92DE
:1057C0009F92AF92BF92CF92DF92EF92FF920F9390
:1057D0001F93CF93DF935C01562E3A016901662334
:1057E00009F45DC0482EEC0130E060E0EE24FF24B7
:1057F000FA9480E000E010E05FE04EE0342E2DE00F
:10580000222E91ED892E96E0992E800E911EF401A4
:1058100070817F707F5FDE0190E0442D41950BC069
:105820005C93223089F0E42EEA0E3F5F9F5F119671
:10583000822F9717D0F4F601E30FF11D208121305C
:1058400079F7882349F45C93F301E60FF11DF080AA
:105850006F5FFC9222E0E7CF5C93F501EE0DF11D46
:10586000808180648083FC92DECF903158F4FE0109
:10587000E90FF11D30829F5F05C0FE01E90FF11DA8
:1058800050839F5F9031C8F3F401808184FD2F869F
:105890000F5F1F4F6096822F051508F4B2CFDF917E
:1058A000CF911F910F91FF90EF90DF90CF90BF901D
:1058B000AF909F908F907F906F905F904F903F90B0
:1058C0002F9008958091BE050E947C14882339F0A2
:1058D000809101068093CD0681E08093460608956D
:1058E0001092AD0584E20E94FF1610927D0480E0C4
:1058F0000E94FF160E940D190E9411180E948B171A
:105900008091FB040E94991780E00E94571E089521
:1059100081E08093AD0584E20E94C7160E948B1738
:1059200080E00E94991780E00E94571E089510920F
:1059300048060E9411180E948B170E940D19809131
:10594000FB040E9499171092440681E20E94FF1600
:1059500080E00E94571E109234078CEF0E94AD1019
:1059600008951092BD0581E08093440681E20E9473
:10597000C71680E00E94571E80914404882321F4BA
:105980008091450480FDFCCF109245041092610483
:105990001092A2048091A2048093A40481E08093D9
:1059A0004806809334078AEF0E94AD1008958091D5
:1059B0008E04882311F480E0089581E00E94A514EC
:1059C000882321F081E080938F04089581E00E9474
:1059D0006614882381F380E00E945014882359F3D1
:1059E00082E080938F0481E0089588E00E94501443
:1059F000882369F09091CD0688E08093BE0590934E
:105A0000010683E08093CD0681E0809346060895E9
:105A100080914404823011F080E008950E94DC10EF
:105A20008093290780E00895AF92BF92CF92DF92D2
:105A3000EF92FF920F931F93CF93DF935B01C82EDA
:105A4000DD24C294D29450EFD522DC24C522DC247C
:105A5000EE24C0E0D0E0FF24F39405C02196F39437
:105A6000F1E1FF16B1F085010C0F1D1FC6018C0F6F
:105A70009D1F0E94661FF8018083EE2079F78081C8
:105A80008F708E3059F7EF2C2196F394F1E1FF16C9
:105A900051F7EE20A1F490E1F50187858F708D30EC
:105AA000B9F0892F81508F70DF91CF911F910F91A5
:105AB000FF90EF90DF90CF90BF90AF9008959E2D14
:105AC000915051F791E0F50187858F708D3049F73E
:105AD000903110F08EE1E8CF892F81508F70806176
:105AE000E3CFBF92CF92DF92EF92FF920F931F937B
:105AF000CF93DF936801E82EFF24EE0CFF1CE60E27
:105B0000F11CEE0CFF1CEE0CFF1CEE0CFF1CE40E57
:105B1000F11CE294F29470EFF722FE24E722FE24B7
:105B200030E022953295307F3227207F3227B22E07
:105B3000222379F0C0E0D0E086010C0F1D1FC701C1
:105B40008C0F9D1F0E94661FF80180832196CB1544
:105B500098F3DF91CF911F910F91FF90EF90DF901D
:105B6000CF90BF900895EF92FF920F931F93CF9322
:105B7000DF93182F062F0E94D618E12EFF24EE0C7B
:105B8000FF1CEE0CFF1CEE0CFF1CE00EF11CE2945F
:105B9000F294A0EFFA22FE24EA22FE24C0E0D0E034
:105BA000FE01EA52F94F8081BE016E0D7F1D0E94F9
:105BB000221F2196C031D10599F70E94D618DF9196
:105BC000CF911F910F91FF90EF900895CF92DF92A8
:105BD000EF92FF920F931F93CF93DF93E22E680112
:105BE000082F10E0000F111F060F111D000F111FCD
:105BF000000F111F000F111F040F111D02951295A8
:105C0000107F1027007F1027FF24E294F29480EF8A
:105C1000F822FE24E822FE24FE2C82E00E94C71611
:105C20000E94D618EE2099F0C0E0D0E0F601EC0F0B
:105C3000FD1F8081B8016C0F7D1F0E94221F82E032
:105C40000E94A20F0E94E20C2196CF1578F382E009
:105C50000E94FF160E94D618DF91CF911F910F91DD
:105C6000FF90EF90DF90CF900895EF92FF920F9307
:105C70001F93CF93DF93182F062F0E94D618E12E83
:105C8000FF24EE0CFF1CEE0CFF1CEE0CFF1CE00EC4
:105C9000F11CE294F29440EFF422FE24E422FE246C
:105CA000C0E0D0E0CE018E0D9F1D0E94661FFE0158
:105CB000EA52F94F80832196C031D10599F71092AD
:105CC0007D0480E00E941C170E94D618DF91CF91BE
:105CD0001F910F91FF90EF900895809144048823C5
:105CE00049F40E94C80080914404813049F00E9428
:105CF000FB1308950E94C900809144048130B9F7D4
:105D00000E94021408950F931F938091CE068093F2
:105D1000D50680914A068823C9F0809102068093B7
:105D2000E6068091BA05809327078091BC05809391
:105D3000430680914A068093490610924A06809154
:105D40008004823088F01F910F9108959091270769
:105D50008091BA059817B9F380918004823098F742
:105D60008091BA05809327078091E6066091270706
:105D700040914306209149060DE816E00E94712DDE
:105D8000609143068091CF069091D0060E94AA2A86
:105D90001F910F9108951092340780E00E94571EC2
:105DA0008CEF0E94AD1080914404813011F00E946C
:105DB000D11310928B061092A2048091A2048093BA
:105DC000A4041092BB058DE896E09093D0068093D2
:105DD000CF068091F7048D3031F0833021F08B3085
:105DE00011F0873011F40E94832E80915204882391
:105DF00061F480915104882309F40895809151043D
:105E00000E948710109251040895809152040E94BC
:105E1000871010925204EDCF4F925F926F927F9253
:105E20008F929F92AF92BF92CF92DF92EF92FF92AA
:105E30000F931F93CF93DF9381E08093CD068093E0
:105E4000460610E0C0E0D0E0BB24FF24F394AA246F
:105E5000AA9442E0E42E34E0932E23E0822E90E2D6
:105E6000792E80E1682E0FE0502EB1E14B2E0E947A
:105E700015160E94E20C8091CD06873009F4DFC030
:105E8000883008F07EC0843009F46FC2863009F48F
:105E90002EC2813061F780914606882331F010923E
:105EA00046060E9476170E94D61887E10E94A51424
:105EB000882361F08091CD0697E19093BE05809391
:105EC000010687E08093CD06F092460688E00E94A6
:105ED000A514882361F08091CD0698E09093BE05CB
:105EE0008093010686E08093CD06F092460681E01D
:105EF0000E94A514882351F08091CD06F092BE0532
:105F0000809301069092CD06F09246068EE00E94A4
:105F1000A514882359F09091CD068EE08093BE059C
:105F2000909301065092CD06F092460682E00E94C0
:105F3000A514882351F08091CD06E092BE05809390
:105F400001066092CD06F09246069091F104809190
:105F5000F704891709F48BCF8091F1048093F7043B
:105F6000DF91CF911F910F91FF90EF90DF90CF9035
:105F7000BF90AF909F908F907F906F905F904F9069
:105F80000895803109F42FC1813109F4BEC08F30EA
:105F900009F06DCF80914606882349F0109246069D
:105FA000F09283048091F2048093820410E0809147
:105FB000BE050E947C14882349F0809101068093DD
:105FC000CD06F0924606112309F0DBC20E94491566
:105FD000882369F0982F9150933048F48091B6044B
:105FE000981729F09093B604F092830411E0809101
:105FF000B604813009F48BC280918304882309F4AC
:1060000036CF109283040E947F180E948B178091D4
:10601000B6048F5F0E941F188091B604813009F08A
:1060200026CF8091B90481500E9499170E941516BD
:106030000E94E20C8091CD06873009F021CF80913B
:106040004606882339F010924606F092830480E0D9
:106050000E94C7168091BE050E947C14882351F0CF
:10606000809101068093CD06F092460680918304CC
:1060700081FDD0C20E944915882389F0982F915044
:10608000933068F480914404981749F09093440445
:106090000E946D2E8091830483608093830483E04B
:1060A0000E946614882379F0809186048F5F809324
:1060B0008604809186048170809386048091830495
:1060C00083608093830486E10E946614882309F02C
:1060D000AEC18091830480FFCACE809183048E7FFD
:1060E000809383040E947F18809144048F5F0E94F4
:1060F0001F1883E20E94FF1680918604882309F00E
:106100006FC083E20E94C7166BC080914606882349
:10611000C9F010924606F0928304A0928104809107
:10612000AC04813009F43FC2823009F427C28430C4
:1061300009F421C2883011F48092810482E00E9427
:10614000C71610E08091BE050E947C14882349F098
:10615000809101068093CD06F0924606112309F046
:1061600025C20E944915882341F1982F91509430FF
:1061700020F580918104981701F190938104F092A9
:10618000830480918104882309F06AC241E08091F0
:106190008104823009F46AC280918104833009F459
:1061A0006BC2242F30E0C901880F991F820F931F03
:1061B000880F8093B3044093AC04809183048823B8
:1061C00009F455CE109283040E947F1880918104B7
:1061D000843008F005C2809181048F5F0E941F18EF
:1061E0000E94D61844CE80914606882359F010921A
:1061F0004606F092830410920104F092810410E0AC
:10620000C0E0D0E08091BE050E947C148823B1F0EC
:10621000809101068093CD06F0924606112351F03D
:1062200080918104813009F45DC2809181048230C3
:1062300009F425C210924E04F092010480E00E94FD
:106240006614882361F080918104823041F0E092ED
:10625000810482E20E94E316F092830410E00E941F
:10626000C315282F882389F0CE01880F991F880F26
:10627000991F880F991FCC0FDD1FC80FD91F215000
:10628000C20FD11DE092830411E00091810402301D
:1062900009F459C180918304882309F4E8CD8091E1
:1062A0008104813009F48CC180918104823009F02D
:1062B000DECD80918304823009F042C20C2F8BE145
:1062C0000E94FF168CE10E94FF16002339F0B7FCF4
:1062D00062C21B141CF48CE10E94C716802F90E050
:1062E0000E942602F0924E0410928304C0CD809149
:1062F0004606882339F010924606109283041092C5
:10630000810410E08091BE050E947C14882349F02E
:10631000809101068093CD06F0924606112309F084
:106320006CC180918104882309F4D9C02091810433
:10633000213009F4B7C020918104223009F486C0CD
:1063400080918304813009F4A2C08091830482305B
:1063500009F08DCD109283040E948B178091BC04AC
:106360000E9499170E94D61882CD809146068823F4
:1063700039F010924606F09283041092810410E0E6
:106380008091BE050E947C14882331F18091010622
:106390008093CD06F09246061123E1F080918104AE
:1063A000882311F4F092810480918104813210F0ED
:1063B000709281049091000280918104981751F0AD
:1063C00080918104809300026091000287E090E058
:1063D0000E948B0210924E040E94C315382F88230E
:1063E00089F0809181042AE0829FC001112480936A
:1063F0008104809181048150830F80938104E09215
:10640000830411E080918304882309F430CD9091B6
:10641000000280918304823009F413C1892F90E037
:106420000E942602F0924E041092830420CD909197
:10643000010687E18093BE05909301064092CD0648
:10644000F092460680E00E94FF1643CE9091F2043F
:1064500080918204981759F08091F204809382040D
:1064600020938304809182048093BC0411E089E02E
:106470000E947C14882309F463CF109281048BE17D
:106480000E94FF1680918304813009F05ECF109244
:1064900083040E948B178091CF040E9499170E9459
:1064A000D618E5CC9091F20480918204981759F0A7
:1064B0008091F2048093820420938304809182046B
:1064C0008093CF0411E08AE00E947C14882309F4B1
:1064D00032CF109281048CE10E94FF162CCF8AE00B
:1064E0000E946614882309F0AFC089E00E946614F8
:1064F000882309F41BCF8BE10E94C716E092810428
:10650000E09283048091F204809382040FCF9091F3
:1065100082048091F204981709F46ECD8091F20400
:1065200080938204909182049F5F923008F418C196
:106530008091B904981709F45FCD9093B904F09253
:10654000830411E059CD89E00E946614882331F05C
:106550001B1424F400938304BB24BA948AE00E94A1
:106560006614882309F496CEB7FE94CEE092830495
:10657000BB24B3948FCEE0928104E0CDF0928104ED
:10658000DDCD8091B9046091B60490E001978295C9
:106590009295907F9827807F9827682B8AE090E0DB
:1065A0000E948B0213CD10928104C8CD8EE090E042
:1065B0006091AC040E948B0282E00E94FF16D1CD54
:1065C00080918304823009F4CDC080919804909129
:1065D00099040E942602F0924E041092830464CE25
:1065E00085E00E941F1886E00E941F1887E00E9425
:1065F0001F1888E00E941F18F3CD83E090E060919F
:10660000CF040E948B0284E090E06091BC040E9461
:106610008B0287CE8091860490E081709070829585
:106620009295907F9827807F9827609144046F709F
:10663000682B82E090E00E948B0280E00E94FF16AF
:1066400019CD90918104EACE8CE10E94C716F09298
:106650008104F09283048091F2048093820445CFF8
:1066600042E080918104823009F096CD44E080912F
:106670008104833009F095CD48E080E39ACDB7FCE2
:1066800081C081E0C536D10508F073C0992787FD28
:1066900090958C9F60018D9FD00C9C9FD00C1124F5
:1066A000BC2C6C2D772767FD7095872F972F22EED6
:1066B00034E040E050E00E94F74960537D4E8C4E3C
:1066C0009F4F0C2DF8946093090270930A028093F7
:1066D0000B0290930C028DE090E0602F0E948B02E1
:1066E0007894A8CDC431D10508F440C081E0CD3202
:1066F000D80710F0CCE2D1E0F89480919804909102
:1067000099048C179D07D1F0D0939904C0939804F5
:1067100080919804909199040E94F10280919804CC
:10672000909199049093B2048093B104609198047D
:106730007091990485E090E00E949502789475CD5F
:106740008DE090E00E948402282F992787FD909584
:1067500097FD1DC0082F27FD17C0BB24B394AFCDF4
:1067600092E0E6CECE010E94260235CFC4E1D0E011
:10677000C3CFC0E0D0E0BB2460ED72E183E190E0E4
:1067800000E0A0CF8FEF7ECFBB24BA9498CD909538
:1067900081959F4FDFCF8BE10E94C7169ACD1F9343
:1067A000DF93CF930F92CDB7DEB780E00E94571EE4
:1067B00010928B061092450410926104109290047E
:1067C00010925A041092A2048091A2048093A4040F
:1067D0001092BB058DE896E09093D0068093CF068B
:1067E000109143060E948A2A898389818F708F5F66
:1067F000809300041093C005898184FD1BC08CE048
:106800008093FF0383E080933407809144048130B8
:1068100011F00E9409148AEF0E94AD1083E080936A
:106820004C0410925104109252040F90CF91DF91BA
:106830001F91089580E1E4CFEF920F931F93982F5B
:10684000882309F495C0813029F080E01F910F91D1
:10685000EF90089580914606882309F0F9C00E94C0
:106860004915882399F1982F915080914A068823E1
:1068700041F4809143068093BC058091E6068093A5
:1068800002068091BC05891770F48091BC05981BA5
:106890009F5F90934A0680914A06853008F446C16E
:1068A00084E080934A0680913407882309F441C12B
:1068B00080914306609149064091BC0520914A06AB
:1068C0000091C005E090BA050E94C51984E10E94BC
:1068D0006614882309F0DEC085E10E9466148823CF
:1068E00009F0CEC080913407882321F590912707C5
:1068F0008091BA059817F1F08091BA058093270727
:106900008091E60660912707409143062091490651
:106910000DE816E00E94712D8091430660914906B2
:106920004091BC0520914A060091C005E090BA054F
:106930000E94C51980913407882329F480914A0662
:10694000882309F0D4C00E946315982F882309F486
:106950007CCF809181049150981709F076CF809177
:1069600001068093CD0681E08093460680E06ECFDD
:106970000E944915982F8823D1F584E10E9466145E
:10698000882309F49FC01092BA0588E00E94C716B8
:1069900081E00E94FF1680913407882309F055CFCB
:1069A000909127078091BA05981709F44ECF8091EE
:1069B000BA05809327078091E606609127074091EA
:1069C0004306209149060DE816E00E94712D809142
:1069D0004306609149064091BC0520914A0600910A
:1069E000C005E090BA050E94C51980E02FCF8091C4
:1069F000FC048093020601E000934A06192F11500F
:106A00001093BC0584E10E945014882309F44BC004
:106A10001092BA0588E00E94C71681E00E94FF1616
:106A2000109381048091CD06809301068DE08093C0
:106A3000CD0681E0809346061092CE068091340701
:106A4000882309F44FC081E01F910F91EF900895C2
:106A50001092460690938E048091430660914906F9
:106A60004091BC0520914A060091C005E090BA050E
:106A70000E94C5190E944915882309F427CFF3CE37
:106A800081E08093BA0588E00E94FF1681E00E94B1
:106A9000C71628CF1092BA0588E00E94C71681E079
:106AA0000E94FF1619CF85E10E945014882309F433
:106AB000B7CF0093BA0588E00E94FF1681E00E94DC
:106AC000C716AECF85E10E946614882309F463CF10
:106AD00081E08093BA0588E00E94FF1681E00E9461
:106AE000C71659CF82E00E94792A81E0ADCF80910C
:106AF00002068093E6068091BA058093270780916D
:106B0000BC058093430680914A0680934906109203
:106B10004A068091E606609127074091430620913E
:106B200049060DE816E00E94712D0DCF80914A06AE
:106B3000B8CE809102068093E6068091BA058093D4
:106B400027078091BC058093430680914A06809375
:106B5000490610924A068091E60660912707409107
:106B60004306209149060DE816E00E94712DA0CE43
:106B70002F923F924F925F926F927F928F929F924D
:106B8000AF92BF92CF92DF92EF92FF920F931F933B
:106B9000DF93CF930F92CDB7DEB70E9415161092F8
:106BA000CE068091CE068093D50680913407882347
:106BB00011F40C94913F84E08093CD0681E08093A2
:106BC00046066624992488245524772473945CE02F
:106BD000452E43E0342E34E0232E0E9415160E94E9
:106BE000E20C1091CD061830E9F0193008F04EC0D3
:106BF000153009F4A5C4163008F096C0113009F418
:106C00002FC2143009F413C40E94082D882329F7D9
:106C10000E94D72C0E9415160E94E20C1091CD06FE
:106C2000183019F780914606882349F010924606DD
:106C30000E94761783E20E94C716709280048091AA
:106C4000BE050E947C148823A1F0809101068093E8
:106C5000CD0670924606109280048091E6066091FF
:106C6000270740914306209149060DE816E00E944F
:106C7000712D0E944915882309F013C50E946315E0
:106C8000882311F281500E94BD19BECF1B3009F438
:106C9000E1C21C30C0F5193009F481C21A3009F084
:106CA000B3CF809146068823F1F01092460680E02B
:106CB0000E94C7160E94D6188091E60660912707A9
:106CC00040914306209149060DE816E00E94E62D0A
:106CD00080E00E94FF160E94D6182092CD06709286
:106CE00046061092800480918304882331F020921C
:106CF000CD067092460610928304809183048F5FC4
:106D00008093830481CF1C3009F47AC11D3009F0CF
:106D10007BCF81E00E941C348091CD068D3009F438
:106D200073CF10928E0470CF163009F4F9C017306B
:106D300009F06ACF80914606882389F110924606B1
:106D40000E947617609149068DE896E047EE56E07E
:106D500021EC35E00E94F82A80E00E94C7161092CC
:106D6000830489E080938104109282048091490613
:106D7000882391F020E0E22FF0E0EF52F94F90816C
:106D8000809182048F5F9F70890F809382042F5FB0
:106D900080914906281778F366249924552480E0C9
:106DA0000E94A514882311F06624639488E00E9451
:106DB000A514882311F082E0682E87E10E94A514B3
:106DC000882311F003E0602E80918104893009F45A
:106DD00024C780918104813009F4F8C68091810430
:106DE000882309F42CC580918104882329F080919F
:106DF0008104807F09F45CC0109181048EE00E94C0
:106E00006614882351F0809181048061809381040D
:106E1000F5E0F0938304B2E05B2E8FE00E946614ED
:106E2000882351F08091810480628093810485E001
:106E3000809383045524539484E10E94661488232C
:106E400049F08091810480648093810495E090935F
:106E5000830455248EE00E947C14882339F08091AD
:106E60008104807E80938104209283048FE00E94BD
:106E70007C14882339F080918104807D8093810483
:106E80002092830484E10E947C14882339F080914D
:106E90008104807B80938104209283048091830409
:106EA000853009F48BC580918304843009F476C55C
:106EB00080918104883009F469C48091830490E052
:106EC00083709070892B09F079C4662009F49CCEF8
:106ED000609149068DE896E047EE56E021EC35E0FA
:106EE0000E94D92B8091E6066091270740914306C6
:106EF000209149060DE816E00E94E62D81E0681613
:106F000009F46FC592E0691609F474C0F3E06F16D6
:106F100009F07ACE87E08093CD067092460674CE53
:106F2000809146068823D9F0109246060E94761773
:106F3000609149068DE896E047EE56E021EC35E099
:106F40000E94F82A84E20E94C716109283041092CD
:106F50008204F3E6F093810466249924882480E077
:106F60000E94A514882311F06624639488E00E948F
:106F7000A514882311F022E0622E809181048336CB
:106F800009F419C680918104813009F4B5C5809156
:106F90008104833009F43DC580918104882309F47C
:106FA0008FC48091830490E083709070892B09F0E6
:106FB00057C4662009F428CE609149068DE896E012
:106FC00047EE56E021EC35E00E94D92B8091E60691
:106FD0006091270740914306209149060DE816E08D
:106FE0000E94E62D81E0681609F4FBC492E0691660
:106FF00009F00ACEE6E0E093CD067092460604CE94
:1070000080914606882389F01092460690917E046E
:1070100080914906981709F4B3C670928304809151
:1070200001068093CD06709246068091BE050E94AF
:107030007C14882309F4E8CD809101068093CD0665
:107040007092460680918304882309F429C68DE056
:107050000E94FF1682E00E94FF160E94D618D4CD2F
:10706000809146068823E9F01092460680E00E944F
:1070700062020E94761782E20E94C71610938E0465
:1070800081E20E94FF16809143066091490640917B
:10709000BC0520914A0600914306E090BA050E9483
:1070A000C51980E00E941C3480E00E946614882389
:1070B00029F085E08093CD067092460683E00E9419
:1070C0006614882359F08091CD063092BE058093D6
:1070D000010688E08093CD067092460688E00E9403
:1070E000A514882329F096E09093CD067092460669
:1070F00087E10E94A514882329F0E7E0E093CD06FC
:10710000709246068BE00E94A514882359F0909156
:10711000CD068BE08093BE05909301068093CD064B
:10712000709246068DE00E94A514882359F0909134
:10713000CD068DE08093BE05909301064092CD066A
:10714000709246068091CD06813011F010928E0427
:1071500080913407882321F02092CD067092460654
:107160009091F1048091F704891709F44DCD809135
:10717000F1048093F7040F90CF91DF911F910F914D
:10718000FF90EF90DF90CF90BF90AF909F908F9047
:107190007F906F905F904F903F902F9008958091D7
:1071A0004606882381F01092460682E20E94FF166E
:1071B00081E00E94571E80E00E94571E80E00E94DE
:1071C000620270928E0480913407882309F4C1C250
:1071D000909181048091BF059817C9F09090810427
:1071E0008091BF058093810480918304833009F4EA
:1071F000E4C580918304823050F08091B9058823E2
:1072000031F4E0918104F0E0EF53FA4F708286E1AF
:107210000E946614882329F08091B905882309F417
:1072200007C580918304833009F4E0C386E10E949E
:107230007C14882309F4E8CC80918304823009F01F
:10724000E3CC7092830480E00E94571E82E00E948B
:10725000FF16DACC80914606882361F0109246062C
:1072600082E20E94FF168FE00E94C7160E94D61885
:10727000109283048091BE050E947C14882309F437
:1072800042C0809101068093CD067092460680919F
:107290008304882391F58091E60630912707209199
:1072A000430690E0880F991F830F911D880F991F47
:1072B000880F991F880F991F280F20937F048091B2
:1072C000490680937E048823C1F090E0A0E0B0E0FE
:1072D000282F30E022953295307F3227207F3227C9
:1072E000FD01E357F94F8081AD5FB94F8C939F5FEC
:1072F000A92FB0E0A217B3079CF38FE00E94FF16FE
:107300008DE00E94FF168DE00E946614882309F428
:107310007BCC80918304882309F076CC80917E0415
:10732000882309F471CC709283048091E606209141
:1073300027071091430690E0880F991F820F911D37
:10734000880F991F880F991F880F991F180F809118
:107350007F04181709F458CC8DE00E94C71682E00C
:107360000E94C7160E94D61890917F04809149060A
:10737000882309F442C0A92EBB24A294B294B0EF92
:10738000BB22BA24AB22BA247501C12EDD24C294DB
:10739000D294A0EFDA22DC24CA22DC2400E010E040
:1073A000C7010E94661F882E0357194FF80180837A
:1073B000C6010E94661FB7010E94221F882DB601D8
:1073C0000E94221F82E00E94A20F0E94E20C0894F9
:1073D000E11CF11C0894C11CD11C8E2D8A19082FA8
:1073E00010E08091490690E082959295907F9827D1
:1073F000807F9827081719079CF2109143068DE8A3
:1074000096E00E948A2A898389818F708F5F80939A
:1074100000041093C005898184FD8DC58CE08093A4
:10742000FF0382E00E94FF160E94D618EDCB8091E8
:1074300046068823E9F0109246060E94761782E2FB
:107440000E94C71670928E0481E20E94C716809136
:107450004306609149064091BC0520914A0600917F
:107460004306E090BA050E94C51981E00E946202BD
:1074700083E00E94A514882309F445C080914A0640
:10748000882309F06AC4909127078091BA0598175C
:1074900081F08091BA05809327078091E60660917C
:1074A000270740914306209149060DE816E00E9407
:1074B000712D609149068DE896E047EE56E021EC8B
:1074C00035E00E94F82A80E090E0FC01EF53FA4F8B
:1074D0001082019680349105C1F782E08093800488
:1074E00010922A0710928204109281041092830451
:1074F0001092B9057092850489E08093CD06709250
:10750000460699249A948091CD06843011F0109209
:107510008E0480913407882321F47092CD067092F6
:10752000460680918D04813009F06ECB10928D0457
:107530009091F1048091F704891709F018CE64CB7B
:10754000809146068823C9F0109246060E9476175D
:10755000709283048DE896E00E948A2A282F2F706B
:107560002F5F2093810490E0929582958F708927F8
:107570009F7089278170809382048EE00E94E415B9
:10758000823009F4D9C08AE00E94E415823009F4FF
:10759000B9C089E00E94E415823009F4C1C08FE0CF
:1075A0000E946614882391F03092830480918204B3
:1075B000882311F440928104809182048F5F80932C
:1075C000820480918204817080938204809183047C
:1075D00080FF21C080918304815080938304809137
:1075E0008204882309F4CEC180918104803108F49B
:1075F000DEC381E08093810483E00E94C7168091FE
:107600008104882309F0BBC181E0809381048091CB
:1076100081040E94AF1780E00E947C14882309F443
:10762000F3CA809183048230B8F182E080938004B1
:107630008DE896E061E047EE56E021EC35E00E94EF
:10764000F82A9091810480918204811180E1915007
:107650009F70892B8093D1068DE896E061E047EE1C
:1076600056E021EC35E00E94D92B8091E60660912E
:1076700027074091430621E00DE816E00E94E62D21
:107680008091E606609127074091430620914906C4
:107690000E94712D109280047092CD067092460661
:1076A000B3CA182F1150812F0E94B5198091E60698
:1076B00090912707E82EFF24EE0CFF1CE90EF11C29
:1076C000EE0CFF1CEE0CFF1CEE0CFF1CE10EF11C7F
:1076D000E294F29470EFF722FE24E722FE24870161
:1076E000005F1F4F8FE0B7010E94221F82E00E94BF
:1076F000A20F0E94E20C0894E11CF11CE016F106B6
:1077000089F7BCCA809181048F708F5F8093810458
:107710003092830489E00E94E415823009F03FCF63
:107720008091810490E00E968F7090708F5F8093AF
:1077300081043092830433CF80918304823008F433
:10774000B8C3809181048F5F809381043092830459
:107750001ACF81E00E94571E80E00E94571E1092AF
:1077600085041092A4047092CD0670924606109281
:1077700080048091E606609127074091430620919E
:1077800049060DE816E00E94712D22CDE92DF0E0AA
:10779000EF53FA4F5082939480918204981610F020
:1077A0006624639470928304109281048091830410
:1077B00090E083709070892B09F487CB0E948B171F
:1077C000809149068823B1F090E080E001C08E2FBF
:1077D000E92FF0E0EF52F94FE081EF70EF5FE80F33
:1077E000981618F09E1608F4F1C29F5F8091490622
:1077F000981768F384E00E94FF1683E00E94FF164A
:1078000088E00E94FF168091830480FD13C0E2E0AF
:107810005E1609F492C3F1E05F1609F492C3552095
:1078200031F084E00E94C71683E00E94C71688E00A
:107830000E94C7160E94D6181092830446CB86E198
:107840000E94A514882309F4CECAE92DF0E0EF5375
:10785000FA4F50807092810482E080938304C3CAFF
:107860000E948B17E92DF0E0E55BF94F80818F3F97
:10787000D1F0108112951F7000810F70010F0F5F02
:10788000101738F010C0812F0E94CD171F5F1017FE
:1078900050F48091830480FDF6CF812F0E949917C8
:1078A0001F5F1017B0F38091830480FFF4C1882D0F
:1078B00060E00E94201A109283040E94D61879CBAF
:1078C00086E10E946614882309F08AC20E94FB1494
:1078D000882309F0BCC287E10E947C14882329F028
:1078E000FFE39F0E9F22709283048EE00E94661435
:1078F000882321F080E1882A709283048FE00E941F
:107900006614882321F090E2892A7092830484E12E
:107910000E946614882321F0E0E88E2A7092830486
:1079200085E10E946614882321F0F0E48F2A70928A
:1079300083048EE00E947C14882321F08FEE88223D
:10794000709283048FE00E947C14882321F09FEDC5
:1079500089227092830484E10E947C14882321F0A0
:10796000EFE78E227092830485E10E947C148823C5
:1079700009F417CBFFEB8F227092830412CB809116
:10798000810443CE80918104813108F413C281E0E7
:107990008093810483E00E94FF1631CE112359F0B9
:1079A00080918104882339F49394809182049816FD
:1079B00010F066246394709283047ACA112309F04C
:1079C000EDC180918104882309F4E8C1662029F47F
:1079D000E92DF0E0EF53FA4F508282E08093830468
:1079E00062CA6092CD06609246060EC90E94931547
:1079F000882309F41BCC82E08093830486E10E94F3
:107A00005014882309F012CC709283040E94571EF0
:107A10000DCC0E94FB14182F0E941515882319F411
:107A2000112309F4B9CAE92DF0E0E951F94F808238
:107A300080E00E94571E82E00E94A20F9394FFE311
:107A4000F91518F41092820499247092830410920C
:107A500081048FE088228EE00E945014882311F068
:107A600090E1892A8FE00E945014882311F0E0E20F
:107A70008E2A84E10E945014882311F0F0E88F2AA6
:107A800085E10E945014882311F080E4882A112394
:107A900009F482CA812E8A949FE089228EE00E9496
:107AA0005014882311F0E0E18E2A8FE00E945014D8
:107AB000882311F0F0E28F2A84E10E945014882379
:107AC00011F080E8882A85E10E945014882311F083
:107AD00090E4892AE82DF0E0EF73F070EE5FFB4F41
:107AE000482D4078808160E00E94401E82E08093B3
:107AF00083043092810450CA86E10E947C1488235A
:107B000009F0DCC18EE00E946614882349F0882DBC
:107B1000809580719FEE8922882A82E08093830479
:107B20008FE00E946614882349F0882D809580722A
:107B3000EFED8E22882A82E08093830484E10E9404
:107B40006614882349F0882D80958078FFE78F227E
:107B5000882A82E08093830485E10E94661488234A
:107B600049F0882D809580749FEB8922882A82E0D5
:107B7000809383040E94FB14182F882309F407CAFA
:107B800080E00E94571E82E00E94A20F11501F70D9
:107B9000E0EF8E22812AE82DF0E0EF73F070EE5FC7
:107BA000FB4F482D4078808160E00E94401E82E0BB
:107BB00080938304ECC988E00E947C14882309F434
:107BC000E1C91092810470928304DCC986E10E94AD
:107BD0007C14882319F088E0809381048EE00E9451
:107BE0006614882329F082E08093830412E0512EEA
:107BF0008FE00E946614882329F082E0809383043A
:107C00005524539484E10E946614882309F4E6C83D
:107C100082E0809383045524E1C887E10E947C14AC
:107C2000882309F4D6C81092810470928304D1C8C5
:107C300082E0809383040E947D15882311F03092A6
:107C40008304E0918104F0E0EF53FA4F82E08083F7
:107C5000E0918204F0E0E951F94F8080809247067C
:107C6000E82DF0E0EF73F070EE5FFB4F482D4078A9
:107C7000808160E00E94401E80918104981639F056
:107C800090908104809182048F5F8093820482E0CF
:107C90000E94C716C6CA882D61E00E94201A0BCE2A
:107CA00082E00E94C7160E94D6189091E6062091A5
:107CB00027073091430680917E048823C9F1E92E7D
:107CC000FF24EE0CFF1CE20EF11CEE0CFF1CEE0C70
:107CD000FF1CEE0CFF1CE30EF11CE294F29460EF2B
:107CE000F622FE24E622FE248701A0E0B0E0FD019A
:107CF000ED5FF94F8081A357B94F8C93B8010E9473
:107D0000221F82E00E94A20F0E94E20C0F5F1F4F11
:107D1000802F8E19A82FB0E080917E0490E082958C
:107D20009295907F9827807F9827A817B907FCF233
:107D3000109143068DE896E00E948A2A8983898102
:107D40008F708F5F809300041093C005898184FD3C
:107D5000B3C08CE08093FF037AC9809102068093C0
:107D6000E6068091BA05809327078091BC05809331
:107D7000430680914A068093490610924A068DCBAD
:107D8000992309F44AC982E20E94FF168DE00E94FD
:107D9000C7160E94D6181092830447C99394809105
:107DA0008204981608F412CE6624639416CE80914D
:107DB000810420CC80918104EBCD0E947D15882325
:107DC00009F017CA82E08093830413CA992D981B87
:107DD0008091830480FFA1C0892F0E94CD170ACD16
:107DE000E92DF0E0E951F94F80808EE00E945014B7
:107DF000882311F0E0E18E2A8FE00E94501488233E
:107E000011F0F0E28F2A84E10E945014882311F0CF
:107E100080E8882A85E10E945014882311F090E4BC
:107E2000892AE82DF0E0EF73F070EE5FFB4F482DEC
:107E30004078808160E00E94401E82E0809383044D
:107E4000709281040E94FB14882309F444CD882E8B
:107E50008A94EFE08E228EE00E945014882311F065
:107E6000F0E18F2A8FE00E945014882311F080E205
:107E7000882A84E10E945014882311F090E8892A0E
:107E800085E10E945014882311F0E0E48E2AE82D49
:107E9000F0E0EF73F070EE5FFB4F482D407880818B
:107EA00060E00E94401E82E080938304309281044F
:107EB00012CD1092810445CC80E14CCFE92DF0E049
:107EC000E951F94F80828EE00E945014882381F599
:107ED00088248FE00E945014882311F080E2882AC1
:107EE00084E10E945014882311F090E8892A85E1EA
:107EF0000E945014882311F0E0E48E2A80E00E9452
:107F0000571E9394FFE3F91518F4109282049924F4
:107F10007092830410928104F5CD892F0E949917E5
:107F200069CC81E08093CD06809346060C94E135C0
:107F300090E1892ECECF80E172CA84E00E94C716FC
:107F400079CC83E00E94C71675CC0F931F93CF9313
:107F5000DF93EC01442319F18B0150E070E020E045
:107F600030E0F901EF52F94F60816F706F5FD80117
:107F700090E0FE01E50FF11D80818D939F5F5F5FB3
:107F80009617B8F3760F2F5F3F4F005F1F4F2417F0
:107F900040F3872FDF91CF911F910F91089570E0EB
:107FA000872FDF91CF911F910F910895BF92CF92AC
:107FB000DF92EF92FF920F931F93CF93DF936B01AA
:107FC000B42E442369F17C0110E000E0C0E0D0E071
:107FD000C7010E948A2AFE01EF52F94F8083208157
:107FE0002F702F5FD70190E08D91F601E10FF11D09
:107FF00080839F5F1F5F9217B8F3020F219680E185
:1080000090E0E80EF91ECB1518F3802FDF91CF9189
:108010001F910F91FF90EF90DF90CF90BF90089548
:1080200000E0F3CFCF92DF92EF92FF920F931F9376
:10803000DF93CF93CDB7DEB7C054D0400FB6F894DE
:10804000DEBF0FBECDBF109283041092810482E088
:1080500080938004409149068DE896E06E01089473
:10806000C11CD11CB6010E94D63FE82E809182042B
:108070008E1510F010928204809149068823C1F079
:1080800090E030E0E32FF0E0EF52F94F20812F70C5
:108090002F5F80E0E92FF0E0E55BF94F80838F5F91
:1080A0009F5F8217B8F33F5F80914906381750F3FE
:1080B0000E94151680913407882309F4C9C184E011
:1080C0000E94EA2AFF240E9415160E94E20C1091D9
:1080D000CD06113081F01430F1F10E94082D882373
:1080E00091F70E94D72C0E9415160E94E20C109165
:1080F000CD06113081F70E94F02A882309F0F4C0E0
:1081000086E10E94A514882329F0809184048823A5
:1081100009F088C18091CD06813011F010928E0453
:1081200080913407882309F070C10E94352A882382
:10813000A1F210928004C05CDF4F0FB6F894DEBF4E
:108140000FBECDBFCF91DF911F910F91FF90EF90A8
:10815000DF90CF9008950E94F02A882309F037C15C
:1081600010E086E10E94A514882309F0D0C087E1C1
:108170000E94A514882309F0E6C086E10E947C14C1
:10818000882309F0FCC087E10E947C14882309F051
:1081900001C186E10E946614882309F006C18EE0C1
:1081A0000E946614882339F08F2D809580719FEE90
:1081B000F922F82A12E08FE00E946614882339F031
:1081C0008F2D809580729FEDF922F82A12E084E1CC
:1081D0000E946614882339F08F2D809580789FE760
:1081E000F922F82A12E085E10E946614882339F00A
:1081F0008F2D809580749FEBF922F82A12E00E945F
:10820000FB14282F882361F08F2D90E08F709070E1
:108210000D9734F421502F7080EFF822F22A12E0EB
:1082200088E00E946614882309F44AC08F2D90E0EC
:108230008F7090700D970CF4ECC090EFF92200E075
:1082400010E080918204F601E80FF11DF082409168
:108250004906C6016DE876E00E94A53FE82E81E060
:10826000809384040D301105BCF58F2D61E00E94D0
:10827000201A84E20E94C7160E948B17E0918204A4
:10828000F0E0E55BF94F80810E9499170E94D618B3
:108290008091CD06843011F010928E0480913407C5
:1082A000882309F4AEC080918D04813009F015CF88
:1082B00010928D040E94352A882309F40ECF39CFFD
:1082C000123009F4C9C0113019F70F2D10E00F70EA
:1082D00010700D3011054CF28F2D60E00E94201AB5
:1082E00084E20E94FF16C8CF0E94761782E20E94A5
:1082F000C71610938E0481E20E94FF1680918404B9
:10830000882309F4A1C082E00E94E316F9CE80918F
:1083100082048F5F80938204809182046E2D0E947C
:10832000164A9093820480918204F601E80FF11DB1
:10833000F08082E00E94C71611E087E10E94A51438
:10834000882309F41ACF809182046E2D70E090E0AA
:108350000197860F971F0E94364A8093820480916E
:108360008204F601E80FF11DF08080E00E94C7163C
:1083700011E086E10E947C14882309F404CF82E096
:108380000E94FF160E94D61887E10E947C14882361
:1083900009F4FFCE80E00E94FF160E94D61886E105
:1083A0000E946614882309F4FACE80E00E945014DB
:1083B000882309F4F4CE8091BF05809382048091D4
:1083C0008204F601E80FF11DF08011E0E8CE0E9472
:1083D000761782E20E94C71681E080938E0481E2C4
:1083E0000E94C716809184048823C1F082E00E9415
:1083F000E31680918204F601E80FF11DF08011E090
:10840000B0CE81E00E94EA2A4ECF84E00E94EA2AA0
:108410008CCE8FE0F82E0FE010E013CF82E00E94A8
:10842000FF16E7CF82E00E94FF168091E60660917A
:10843000270740914306209149060DE816E00E9467
:10844000E62D1092840466CE82E00E94FF1658CE7C
:1084500081E00E94EA2A36CE0F2D10E00F701070D6
:10846000F0CE3F924F925F926F927F928F929F9247
:10847000AF92BF92CF92DF92EF92FF920F931F9332
:10848000DF93CF93CDB7DEB7C058D0400FB6F89486
:10849000DEBF0FBECDBF109283041092810482E034
:1084A0008093800440914906B1E4CB2ED12CCC0EB0
:1084B000DD1E8DE896E0B6010E94D63FF82E0E94A0
:1084C000151680913407882309F459C684E00E9468
:1084D000EA2A772444246624552488248A949924FB
:1084E000332433945E010894A11CB11C0E9415161C
:1084F0000E94E20C1091CD061F30B9F0103108F047
:108500008AC0113009F4BAC2143009F44EC20E9474
:10851000082D882359F70E94D72C0E9415160E9417
:10852000E20C1091CD061F3049F70E94F02A8823F3
:1085300009F09BC40E94622C86E10E946614882385
:1085400009F08AC489E00E946614882309F0D5C224
:108550008AE00E946614882309F0C7C286E10E945F
:108560007C14882309F0BDC289E00E947C14882312
:1085700009F0B3C28AE00E947C14882309F0A9C2E2
:108580008DE00E946614882329F080917E04882360
:1085900009F05AC591E0791609F4DBC3A2E07A1616
:1085A00009F4D3C3B3E07B1609F0B1CF3092840451
:1085B000662D70E0842D992787FD9095860F971F73
:1085C000850D911D0E94364A582EFF2099F020E01B
:1085D00030E0F601E20FF31F852D820F662D0E9419
:1085E000164AD501A90FB11D8C9180832F5F3F4F93
:1085F0002F1578F340914906C6016DE876E00E9498
:10860000A53F409149068DE896E0B6010E94D63F0D
:10861000F82E77247CCF113109F41BC1113108F4F5
:1086200080C0123109F073CF0E94F02A882309F02C
:1086300056C40E94622C8CE00E946614882309F0C4
:1086400077C38CE00E947C14882309F06DC38EE010
:108650000E946614882309F05DC38FE00E946614AF
:10866000882309F04DC384E10E946614882309F031
:108670003DC385E10E946614882309F02DC388E07C
:108680000E946614882309F01DC38EE00E947C14AA
:10869000882309F0EFC28FE00E947C14882309F040
:1086A000F2C284E10E947C14882309F0F5C285E1BE
:1086B0000E947C14882309F0F8C288E00E947C1490
:1086C000882309F0FBC2772009F421CF309284047B
:1086D000FF2009F48FCF860110C00E97F9F08E2D80
:1086E0008821D8019C919921892BF80181938F01D0
:1086F0008E2F8C198F1508F07DCF0E941B01E82E5C
:1087000090E08F7090708D30910539F7E7EFEE2291
:108710008E2D90E08F7090700E9709F7F7EFEF2293
:10872000DECF0E94F02A882309F09EC20E94622CAC
:108730008CE00E946614882309F0E7C187E10E945B
:108740006614882309F0ECC180E00E946614882337
:1087500009F0F1C18CE00E947C14882309F0F6C175
:1087600087E10E947C14882309F0F9C180E00E940F
:108770007C14882309F0FCC18EE00E9466148823D3
:1087800009F0FFC18FE00E946614882309F008C237
:1087900084E10E946614882309F011C285E10E94D9
:1087A0006614882309F01AC288E00E9466148823A0
:1087B00009F023C28EE00E947C14882309F02CC2A9
:1087C0008FE00E947C14882309F02FC284E10E946C
:1087D0007C14882309F032C285E10E947C1488232E
:1087E00009F035C288E00E947C14882309F038C261
:1087F000772009F48CCE30928404E2E07E1609F4EE
:10880000D0C3F4E07F1609F46FC4B1E07B1609F021
:108810002CC4FF2009F4EECE860107C00F5F1F4F66
:10882000802F8C198F1508F0E5CE0E941B01E82ED1
:10883000EFE1E81798F30E941B01D8012C916F2DEE
:108840000E94164AF601E90FF11D80818C93208366
:10885000E5CF0E94F02A882309F0F9C20E94622C19
:108860008CE00E946614882309F0E8C28CE00E9424
:108870007C14882309F0DEC28EE00E9466148823EF
:1088800009F0CEC28FE00E946614882309F0BEC2B0
:1088900084E10E946614882309F0AEC285E10E943B
:1088A0006614882309F09EC288E00E94661488231B
:1088B00009F08EC28EE00E947C14882309F084C2E5
:1088C0008FE00E947C14882309F05FC284E10E943B
:1088D0007C14882309F062C285E10E947C148823FD
:1088E00009F065C288E00E947C14882309F068C200
:1088F0008DE00E946614882329F080917E048823ED
:1089000009F043C0172D10FF02CE3092840411FDF0
:10891000EFC2FF2041F1860106C00F5F1F4F802F7D
:108920008C198F1500F50E941B01E82EBFE3B817C4
:10893000A0F30E941B01E82E90E08F7090708D30A4
:10894000910509F404C30E9709F4FEC29E2D9821E7
:10895000D8018C918921982B9C930F5F1F4F802FFA
:108960008C198F1500F3BEEF7B2240914906C6019A
:108970006DE876E00E94A53F409149068DE896E0BB
:10898000B6010E94D63FF82EC2CD872D8095827009
:10899000B1E07B22782A8DE00E94FF16172D71FC32
:1089A000CBC366240E94D618AECF0E94F02A88233B
:1089B00009F07FC284E00E94A514882309F072C2E6
:1089C00085E00E94A514882309F065C282E10E9417
:1089D000A514882309F058C281E10E94A5148823B8
:1089E00009F04BC286E10E94A514882329F08091EA
:1089F0008404882309F016C387E10E94A514882304
:108A000029F080918404882309F0B2C28091CD06B8
:108A1000843041F010928E0482E00E94FF1682E2C0
:108A20000E94FF1680913407882309F48AC180913F
:108A30008D04813009F06BCD10928D040E94352A8F
:108A4000882309F464CD10928004C058DF4F0FB61C
:108A5000F894DEBF0FBECDBFCF91DF911F910F9174
:108A6000FF90EF90DF90CF90BF90AF909F908F904E
:108A70007F906F905F904F903F9008950E94F02AF2
:108A8000882389F48091CD06813011F010928E04F4
:108A900080913407882309F027C20E94352A882351
:108AA00009F435CDD0CF0E94761782E20E94C71616
:108AB00010938E0481E20E94FF1680918404882323
:108AC00009F4CFC282E00E94E31681E00E946202B4
:108AD000D9CF8CE10E94FF1653CD8BE10E94FF1687
:108AE00049CD82E00E94FF163FCD8CE10E94C7165F
:108AF0007E2C73944424439431CD8BE10E94C7169D
:108B00007E2C739444244A9423CD8EE00E94C71691
:108B10007724739487E10E946614882309F414CEA5
:108B200080E00E94C716F2E07F2E80E00E9466146B
:108B3000882309F40FCE82E20E94C716E3E07E2E5E
:108B40008CE00E947C14882309F40ACE8EE00E94F7
:108B5000FF1687E10E947C14882309F407CE80E089
:108B60000E94FF1680E00E947C14882309F404CE42
:108B700082E20E94FF168EE00E946614882309F4A8
:108B800001CE84E00E94C71674E0772E60E1862E45
:108B90005FEE952E8FE00E946614882309F4F8CDCD
:108BA00083E00E94C71644E0742E30E2832E2FED3E
:108BB000922E84E10E946614882309F4EFCD88E0A8
:108BC0000E94C71694E0792E80E8882E0FE7902E39
:108BD00085E10E946614882309F4E6CD81E00E94B5
:108BE000C71614E0712EB0E48B2EAFEB9A2E88E0FE
:108BF0000E946614882309F4DDCD84E20E94C71622
:108C0000F4E07F2EEFE08E2E70EF972E8EE00E9424
:108C10007C14882309F4D4CD84E00E94FF168FE0F1
:108C20000E947C14882309F4D1CD83E00E94FF16B2
:108C300084E10E947C14882309F4CECD88E00E9450
:108C4000FF1685E10E947C14882309F4CBCD81E0D6
:108C50000E94FF1688E00E947C14882309F4C8CD86
:108C600084E20E94FF16C4CD89E10E94C7167724D2
:108C700044245CCD84E00E94FF168FE00E947C14A7
:108C8000882309F40ECD83E00E94FF1684E10E9440
:108C90007C14882309F40BCD88E00E94FF1685E13F
:108CA0000E947C14882309F408CD81E00E94FF16FD
:108CB00088E00E947C14882309F405CD84E20E9498
:108CC000FF1601CD84E20E94C716772473942FE02B
:108CD000822E90EF992ED9CC81E00E94C71677247E
:108CE000739440E4842E3FEB932EC9CC88E00E941D
:108CF000C7167724739460E8862E5FE7952EB9CC6B
:108D000083E00E94C71677247394E0E28E2E7FEDF5
:108D1000972EA9CC84E00E94C71677247394A0E113
:108D20008A2EFFEE9F2E99CC8EE00E94FF168FCCEC
:108D30008EE00E94C7167724739488248A9499241D
:108D400080CC81E00E94EA2A72CE442009F02ECC29
:108D5000DECB442009F4DBCB70928404FF2089F041
:108D6000342D3F0DD60120E0822F830F6F2D0E94FE
:108D7000164AF501E90FF11D8D9180832F5F2F15A4
:108D800098F340914906C50138CC83E00E94FF1654
:108D900084E10E947C14882309F49ECD88E00E941F
:108DA000FF1685E10E947C14882309F49BCD81E0A5
:108DB0000E94FF1688E00E947C14882309F498CD55
:108DC00084E20E94FF1694CD84E00E94FF1678CDC5
:108DD00084E20E94C716A1E07A2A1FE0812EB0EF3C
:108DE0009B2E68CD81E00E94C71691E0792A80E42D
:108DF000882E0FEB902E58CD88E00E94C71681E098
:108E0000782A20E8822E9FE7992E48CD83E00E94A1
:108E1000C716F1E07F2A40E2842E3FED932E38CD35
:108E200084E00E94C716E1E07E2A60E1862E5FEEB4
:108E3000952E28CD8EE00E94FF161ECD8EE00E945A
:108E4000C716B1E07B2A88248A9499240FCD8CE040
:108E50000E94C716772402CD82E00E94C716409078
:108E6000BF054194772473946DCB80E20E94C716AE
:108E700077244424EE2455245DCB6091CD0681E116
:108E800041E10E94D62AAECD6091CD0682E142E159
:108E90000E94D62AA1CD6091CD0680E145E00E94D6
:108EA000D62A94CD6091CD068FE044E00E94D62A68
:108EB00087CD0E94761782E20E94C71630928E04F8
:108EC00081E20E94C71680918404882309F4A6C019
:108ED00082E00E94E31681E00E9462026BCD8BE08B
:108EE0000E94C7167724A5CB84E00E94EA2AD5CD3C
:108EF000FF2009F438CD860107C00F5F1F4F802F78
:108F00008C198F1508F02FCD0E941B01E82EEFE37E
:108F1000E81798F30E941B01662D0E94164AF5017E
:108F2000E90FF11DE0808E2D90E08F7090708D30F4
:108F30009105B9F00E9791F09E2D9821D8018C9152
:108F40008921982B9C93D9CFF7EFEF22FFCCE7EF45
:108F5000EE228E2D90E08F709070F5CC87EFE82296
:108F6000EBCFF7EFEF228E2D90E08F709070E2CF75
:108F700082E00E94FF168091E606609127074091EB
:108F80004306209149060DE816E00E94712D40919C
:108F90004906C801B6010E94D63FF82E10928404FB
:108FA00035CD6F2D6695D9F09F2D915040E050E062
:108FB000A92FB0E09501240F351FF601EA0FFB1F22
:108FC0008081F9018083AA0DBB1DF601E40FF51F16
:108FD00080818C9391504F5F5F4F461748F3FF207D
:108FE00009F408CB81E040E050E06F2D0E94164A62
:108FF000D601A40FB51FF501E90FF11D20812074E2
:10900000F501E40FF51F80818F7B282B2C93892F8E
:109010008F5F4F5F5F4F4F1540F3ECCA82E00E94B5
:10902000FF1659CF82E00E94FF168091E6066091FC
:10903000270740914306209149060DE816E00E945B
:10904000E62D10928404D8CCE39481E0E8228DE0F0
:109050000E94FF16EE2009F07BC066240E94D618FD
:1090600099CA82E00E94FF1630CD609149068DE8D2
:1090700096E0A60121EC35E00E94F82AF82E88231C
:1090800011F1860106C00F5F1F4F802F8C198F15BD
:10909000D0F40E941B01E82EBFE3B817A0F30E9492
:1090A0001B01F80120816F2D0E94164AF601E90F7D
:1090B000F11D8081D8018C9320830F5F1F4F802F7B
:1090C0008C198F1530F3609149068DE896E0A60162
:1090D00021EC35E00E94D92B409149068DE896E0BD
:1090E000B6010E94D63F86CAFF2009F483CA8601D2
:1090F00007C00F5F1F4F802F8C198F1508F07ACA99
:109100000E941B01E82E8FE38E1598F30E941B012D
:10911000D8012C916F2D0E94164AF601E90FF11D1E
:1091200080818821992D9223892B8C93808189219C
:109130002821822B8083DDCF8DE00E94C71683E03B
:1091400096E0B50140917E040E94D63F682E2ACC5D
:109150008DE00E94C71683E096E0B50140917E0441
:109160000E94D63F682E409149068DE896E0B601F0
:109170000E94D63FF82EA3E07A2E44246FCF81E0E0
:109180000E94EA2AA6C9EF920F931F930E94151618
:1091900080913407882309F426C184E00E94EA2ADA
:1091A00007C0113009F47EC00E94082D8823E1F029
:1091B0000E9415160E94E20C1091CD061330F1F0BA
:1091C000143078F3143009F447C01D3069F781E09A
:1091D0000E941C348091CD068D3031F310928E04A4
:1091E0000E94082D882321F70E94D72C0E94151673
:1091F0000E94E20C1091CD06133011F70E94F02A64
:10920000882309F09AC00E94622C882321F01092D2
:10921000800410928E040E94FB14882309F07AC007
:1092200080913407882309F0BFCF86E10E9466143D
:10923000882309F4B9CF80E00E94571E81E00E9484
:10924000A20F80E20E94CE2A9091D506890F60E09D
:1092500040E00E94401EA8CF0E94F02A882309F017
:1092600081C080E00E941C34882309F478C080917A
:10927000CD06843011F010928E048091340788233B
:1092800009F48DC080918D04813009F08DCF10924A
:109290008D040E94352A882309F486CF1F910F91EF
:1092A000EF9008950E94F02A882309F07CC080E0A6
:1092B0000E941C34182F86E10E9466148823C9F48A
:1092C0001123A1F08091CD06813011F010928E040F
:1092D00080913407882309F082C00E94352A8823B0
:1092E00009F462CF1F910F91EF9008950E94F52C21
:1092F000E9CF80E00E94571E81E00E94A20F80E229
:109300000E94CE2A9091D506890F60E040E00E942D
:10931000401ED6CF182F11500E94B618812F0E94E0
:109320008D181093CE0680913407882309F078CFEA
:109330008091CE068093D50673CF0E94761711E0F8
:109340001093800481E00E94620284E20E94C716AA
:109350008091CE060E948D1810938E0454CF0E94E7
:10936000F52C85CF0E94761782E20E94C71681E015
:1093700080938E0481E20E94C7168091430660911B
:1093800049064091BC0520914A0600914306E090B1
:10939000BA050E94C51981E00E94620262CF81E095
:1093A0000E94EA2A6FCF0E94761782E20E94C716B7
:1093B00010938E0481E20E94FF1680914306609113
:1093C00049064091BC0520914A0600914306E09071
:1093D000BA050E94C51981E00E94620268CF84E04C
:1093E0000E94EA2A7ACF81E00E94EA2AE1CE629FB7
:1093F000D001739FF001829FE00DF11D649FE00D8D
:10940000F11D929FF00D839FF00D749FF00D659FED
:10941000F00D9927729FB00DE11DF91F639FB00DEC
:10942000E11DF91FBD01CF0111240895991B79E0B9
:1094300004C0991F961708F0961B881F7A95C9F7E4
:1094400080950895AA1BBB1B51E107C0AA1FBB1F33
:10945000A617B70710F0A61BB70B881F991F5A95C0
:10946000A9F780959095BC01CD01089597FB092E31
:1094700007260AD077FD04D0E5DF06D000201AF4D5
:10948000709561957F4F0895F6F7909581959F4F60
:109490000895A1E21A2EAA1BBB1BFD010DC0AA1F35
:1094A000BB1FEE1FFF1FA217B307E407F50720F04D
:1094B000A21BB30BE40BF50B661F771F881F991FC8
:1094C0001A9469F760957095809590959B01AC0111
:0A94D000BD01CF010895F894FFCF0D
:1094DA0001FFFFFFFFFFFFFFFFD012130000060C82
:1094EA0012000A101A000100010001000100010027
:1094FA00010001000100010001000100010001C09A
:10950A0000800040007F206430480F0405060711E0
:10951A001210130E04050607111210130409050A86
:10952A0006070B110C120D101325212326272422BE
:10953A00201D1E1B191F1C1A1012180F110C130EB6
:10954A000B140D0A1516091704050803060107006E
:10955A00020320191A180C0B0A0904080120191A07
:10956A00180C0B0A092221252320191A18241B1C5E
:10957A000F0E0D04030A0C0B0908010200201B1927
:10958A001C1A180F0C0E0B0D0A0926271D1E1F1078
:10959A00121113141516170506076E306E783078F7
:1095AA00000100070E091C1B1215383F363124230F
:1095BA002A2D70777E796C6B6265484F4641545309
:1095CA005A5DE0E7EEE9FCFBF2F5D8DFD6D1C4C379
:1095DA00CACD90979E998C8B8285A8AFA6A1B4B369
:1095EA00BABDC7C0C9CEDBDCD5D2FFF8F1F6E3E4D9
:1095FA00EDEAB7B0B9BEABACA5A28F8881869394C9
:10960A009D9A2720292E3B3C35321F181116030438
:10961A000D0A5750595E4B4C45426F686166737428
:10962A007D7A898E878095929B9CB1B6BFB8ADAA88
:10963A00A3A4F9FEF7F0E5E2EBECC1C6CFC8DDDA88
:10964A00D3D4696E676075727B7C51565F584D4AF8
:10965A004344191E171005020B0C21262F283D3AE8
:10966A0033344E49404752555C5B7671787F6A6D58
:10967A0064633E39303722252C2B0601080F1A1D48
:10968A001413AEA9A0A7B2B5BCBB9691989F8A8DB8
:10969A008483DED9D0D7C2C5CCCBE6E1E8EFFAFDA8
:1096AA00F4F30409050A06070B110C120D10130036
:1096BA000100010001000100010001000100010098
:1096CA00010001000100010001C000800040000CFF
:1096DA0001011718191A1B1C1D1E1F202122233FC6
:1096EA003F3F0B0C0D0E0F10111213141516173FD6
:1096FA003F3F232425262728292A2B2C2D2E2F3F8E
:10970A003F3F0B0C0D0E0F10111213141516173FB5
:04971A003F3F1500B8
:00000001FF
